:1051FE0012010002EF020140C62F00600100010201
:10520E00030109021200010100C01409040000008C
:10521E00FF000000000000000000000000AAAAAA83
:10522E00AAAAAAAAAAEEEEEEEEEEEEEEEEFEFFFFB2
:10523E00FFFFFFFFFFFFFFFFFF7FBFDFEFF7FBFD6E
:10524E00FC7EBFDFEFF7FBFD7EFFFFFFFFFFFFFFE3
:04525E00FFFFFFFF50
:102AC9005028A300000000000000000000000000E2
:102AD90000000041289C004128A1004128910042A2
:102AE900288C00005528734E6F7620323220323000
:102AF90032352D31373A31373A323800422896008B
:052B09000041289400CA
:085A580090280AEEF0A3EFF024
:105A6000E4A3F090280CE0FFD390280BE09F748013
:105A7000F890280AE0648098400D7F141260969098
:075A8000280CE004F080DCBB
:015A870022FC
:102EBE009028687406F0A3E4F0902803F0A374122F
:102ECE00F090280774FFF0A37451F0A374FEF090F5
:102EDE0028057406F0A3E4F0902801F0A3F09028E2
:102EEE0003E0FEA3E0FF902801E0FCA3E0FDC39FFA
:102EFE00EC9E503B902805E0FEA3E07802C333CE53
:102F0E0033CED8F92DFFEC3EFE902807E0FBA3E070
:102F1E00FAA3E0F98D828C83122412FD12607C904C
:102F2E002802E004F070B7902801E004F080AF7D35
:102F3E0006E4FF12606F902805A3E0FD7F1012607B
:102F4E006F902805E0FD7F1112606F7B307D107F42
:102F5E0011125CC3902804E02403FF902803E03490
:102F6E0000FEEF7802CEC313CE13D8F9FF90286976
:102F7E00E02FF0902868E03EF0902803E4F0A37470
:102F8E0012F090280774FFF0A37452F0A37410F09F
:102F9E00902868E0FFA3E0902805CFF0A3EFF0E4BF
:102FAE00902801F0A3F0902803E0FEA3E0FF902804
:102FBE0001E0FCA3E0FDC39FEC9E503B902805E092
:102FCE00FEA3E07802C333CE33CED8F92DFFEC3E0C
:102FDE00FE902807E0FBA3E0FAA3E0F98D828C8334
:102FEE00122412FD12607C902802E004F070B7905B
:102FFE002801E004F080AF902805A3E0FD7F1212B7
:10300E00606F902805E0FD7F1312606F7B307D109E
:10301E007F13125CC3902805A3E0FD7F1412606F2E
:10302E00902805E0FD7F1512606F7B307D107F15B7
:10303E00125CC3E4FDFF12606F7B02E4FD7F301271
:10304E005CC37FC87E00125A587B027D027F30021D
:02305E005CC351
:10532200904000E09027FEF0A37408F09028C7E0B8
:1053320030E0047F0180027F02902800EFF0902885
:10534200687406F0A3E4F01230601231FA1244EAF3
:10535200E49027FDF09027FFE0FF9027FDE0FDD3CA
:105362009F5010902800E0FF1216CA9027FDE0041B
:0E537200F080E2122D179027FEE0904000F030
:01538000220A
:055B3C009027FEEFF0D0
:105B4100904000E09027FFF0E4FDFF12606F902786
:105B5100FEE025E0FD7B027F30125CC39027FFE071
:045B6100904000F080
:015B6500221D
:055AB7009027FEEFF056
:105ABC00904000E09027FFF07D0FE4FF12606F90A4
:105ACC0027FEE0C43354E0FD7B607F23125CC3905F
:075ADC0027FFE0904000F0FD
:015AE30022A0
:105D4B00904000E09027FEF0E4FDFF12606F7F3281
:0F5D5B001260629027FEE0904000F0EF5410FFBE
:015D6A002216
:10519700E49027FDF07F14FE125A589028C7E0FFCD
:1051A700C313540190409DF0125D4BEF7040902760
:1051B700FD04F09027FDE0C3940474809480502E82
:1051C700E4FF125B3C9027FDE0FF125AB77F287E71
:1051D70000125A587F01125B3C7F287E00125A58F2
:1051E700125D4BEF70089027FDE004F080C5902713
:0651F700FDE090409CF079
:0151FD00228F
:103CD6009028CBE0607730E00D54FEF090286DE040
:103CE6004401F0125F269028CBE030E50854DFF05F
:103CF6007F011234F79028CBE030E60854BFF07FFE
:103D0600021234F79028CBE030E708547FF07F02A8
:103D16001234F79028CBE030E10854FDF07F011211
:103D260034F79028CBE030E20854FBF07F021234DF
:103D3600F79028CBE030E30854F7F07F021234F70F
:103D46009028CBE030E40654EFF01260899028CC3E
:103D5600E0607430E00854FEF07F01124191902833
:103D6600CCE030E10854FDF07F021241919028CC5E
:103D7600E030E20854FBF07F041241919028CCE039
:103D860030E30854F7F07F081241919028CCE030D8
:103D9600E40854EFF07F101241919028CCE030E512
:103DA6000854DFF07F201241919028CCE030E608DD
:103DB60054BFF07F401241919028CCE030E7085480
:0C3DC6007FF07F80124191E4FF020B327D
:10377200904000E09027FDF0E4904000F09028EEA9
:04378200E030E768E4
:103786007B017A2679809027FEEBF0A3EAF0A3E985
:10379600F01223F9645A70469027FEE0FBA3E0FA84
:1037A600A3E0F990000112241264B0703190000277
:1037B60012241264CA702790000312241264FE7049
:1037C6001D900003122451900002E412245190002F
:1037D60001E4122451E412243F122EBE8003124B40
:0837E600209028EEE0547FF072
:1037EE009028EFE024FE604214604F14605A14607B
:1037FE00642404706C9028EEE0FF54036063EF3095
:10380E00E007E49028F0F0800A9028F0E0FD7F9227
:10381E0012606F9028EEE054FCF09028F0E05477A0
:10382E00603F9028EF7402F080379028F0E0FF128E
:10383E005C089028EF7403F080271258D9EF6021AE
:10384E009028EF7404F08019E4FF125C089028EFC2
:10385E007405F0800C1258D9EF60069028EF7401B1
:10386E00F09028C1E060279028C0E004F070069028
:10387E0028BFE004F0D39028C0E094C49028BFE0A5
:10388E009409400A1247C1E49028BFF0A3F0902794
:06389E00FDE0904000F087
:0138A4002201
:105C7B009028C7E0C31330E0047F0380027F021239
:105C8B005BB89028C7E030E1031251979028E6E00B
:045C9B004410F0229F
:0B60A2009028E6E030E00354FEF022FE
:103ECD00904000E09027FFF0E4FDFF12606F902816
:103EDD00C8E0C4540FFF9027FDF09028D6E0FD30C8
:103EED00E111EF24FCFFE434FFC313EF139027FD22
:103EFD00F08016ED30E212EF24FEFFE434FFC31321
:103F0D00EF139027FDF04408F09028CAE0C4540F39
:103F1D00FFFE9028D9E0FD30E10EEF24FCFFE434E4
:103F2D00FFC313EF13FE8012ED30E20EEF24FEFF00
:103F3D00E434FFC313EF134408FEEE54F0C454F001
:103F4D00FF9027FDE0540F4FF0FD7FA412606F909E
:103F5D0027FDE0FFC454F0A3F0EF902800F0A3E498
:103F6D00F09028D3E0540FFD7FA512606F9028D6F6
:103F7D00E05401700790286DE04404F09028D9E0DA
:103F8D005401700790286DE04410F09028D3E05450
:103F9D00C0FF90286DE0541F4FFD7FA612606F90FB
:103FAD00286EE0541FFD7FA712606F9027FFE090F1
:033FBD004000F0D1
:013FC00022DE
:105E26009028E6E030E0079028EEE04401F01237D3
:0E5E3600721260A29028E6E054FEF0023ECD0B
:1039C600125E9DEF540F9027FDF0125EB99027FE10
:1039D600EFF0902903E014B40B004003023AD190B3
:1039E60039F375F003A4C58325F0C58373023A1431
:1039F600023A32023A3C023AD1023AD1023AD102B2
:103A06003AD1023A4F023A63023A84023AB6902910
:103A160004E020E00B9027FDE064026003023AD147
:103A2600E4902904F09029037402F022125D6B9051
:103A360029037403F022902904E020E103023AD11D
:103A4600E4F09029037408F022125F5A1260F19094
:103A5600286DE054FEF09029037409F02212576E87
:103A6600125E9DEF540F9027FDF0125EB99027FE6F
:103A7600EFF0E4902905F0902903740AF0229027CC
:103A8600FDE0FF64026005EF64017008902905E01F
:103A960004F08008902905E06002E4F0902905E032
:103AA600D39414748094804022902903740BF022DE
:103AB6009028C7E0C31330E0047F0380027F021220
:0B3AC6005BB81260EE9029037401F061
:013AD10022D2
:10063200904000E09027FDF0E4FDFF12606F7F9094
:100642001260629027FEEFF09040ADE004F0EF7090
:1006520003020B3164EE7003020B319027FEE0308F
:10066200E003020B314401FD7F9012606F7F911213
:1006720060629027FFEFF07F92126062902800EF95
:10068200F0A37401F09027FEE012253308C02C0875
:10069200EC2E06C53006D73206F134071E38091291
:1006A2005009265809445A097890098591098FA062
:1006B20009D7D00A4CD20AE8D80AF4D90AFDDA00DE
:1006C200000B299028EEE04402F09027FFE09028EA
:1006D200F0F00208B99027FFE024FE600C046003EA
:1006E200020B291253E0020B2912566F020B2990BA
:1006F20027FFE014601B046003020B29902806A365
:10070200E0FD7F9312606F902806E0FD7F94020B5C
:1007120026902806A3E0FD7F97020B269027FFE094
:1007220064F0700A7D017F9212606F0208B2902716
:10073200FFE0FD7F9312606F9027FFE0FF122533E9
:1007420007850107850207850307850407BF05079B
:10075200BF0607BF0707BF0807E81107E81207E847
:100762001307E814081E80082381083583083A8499
:1007720008428508588708608808738908A88B0092
:100782000008B2EF540FFD540FC4F8540FC868FFAD
:10079200E4C454F048FE9028DBE0FAA3E0540FFBD7
:1007A200EA4EFEEB4FFF9028DBEEF0A3EFF090282D
:1007B200C7E01313540160030208B280579027FF69
:1007C200E0540FC4F8540FC868FFE4C454F048FE64
:1007D2009028DFE0FCA3E0540FFDEC4EFEED4FFF4E
:1007E2009028DFEE806A9027FFE0540FFD540FC47B
:1007F200F8540FC868FFE4C454F048FE9028DBE0C8
:10080200FAA3E0540FFBEA4EFEEB4FFF9028DBEE1B
:10081200F0A3EFF09028D7EDF00208B29028DB8029
:100822001A9028DBE054F3FEA3E0FFEE4404902884
:10083200DB801D9028DB80219028DDE054F3806C62
:100842009028DDE054F3FEA3E0FFEE44049028DD9F
:10085200F0A3EFF0805A9028DDE0440C804E9028FF
:10086200DFE054F3F0A3E0F09028C7E054F7F08003
:100872003F9028DFE054F3FEA3E0FFEE440490280B
:10088200DFF0A3EFF09028DBE01313540364016060
:100892000C9028DDE013135403640170139028C7F1
:1008A200E04408F0800A9028DFE0440CF0A3E0F076
:1008B200E4FD7F9112606FE4FD7F92020B26902788
:1008C200FFE0FD7C0090280C7401F0A37428F0A3D3
:1008D2007400F07B017F2612434B9027FFE0FF7EDE
:1008E20000A3E0FD12512D020B299027FFE0FD7CB1
:1008F2000090284A7401F0A37428F0A37400F07BDE
:10090200017F26123AD2902800E0FD7FA0020B263A
:100912009028EFE0FD7FA012606F902903E0FD7F39
:10092200A1020B269028D5E0FD7FA012606F9028CF
:10093200D4E0FD7FA112606F9028D8E0FD7FA20273
:100942000B269028C7E0FFC313540125E0FEEF54A5
:10095200014EFD7FA012606F9028C8E0FD7FA112BA
:10096200606F9028C9E0FD7FA212606F9028CAE0F4
:10097200FD7FA3020B267F91126062902903EFF0A4
:10098200020B29902903E0FD7FA0020B269027FF8E
:10099200E0FFA3E0FD125914902802EEF0A3EFF05D
:1009A2001259BC902804EEF0A3EFF0902802E0FD6B
:1009B2007FA012606F902802A3E0FD7FA112606FFA
:1009C200902804E0FD7FA212606F902804A3E0FD4E
:1009D2007FA3020B267F91126062EF7F00FEC007A9
:1009E200C0067F92126062EFFDD0E0FED0E04DFFC4
:1009F200902802EEF0A3EFF01260BDAD077FA012C7
:100A0200606F902803E02401FF902802E03400FE8A
:100A12001260BDAD077FA112606F902803E024022F
:100A2200FF902802E03400FE1260BDAD077FA212E3
:100A3200606F902803E02403FF902802E03400FE58
:100A42001260BDAD077FA3020B267F91126062EF99
:100A52007F00FEC007C0067F92126062EFFDD0E009
:100A6200FFD0E04D902802CFF0A3EFF0902802E0F3
:100A7200FEA3E07802C333CE33CED8F9FF1260BDB5
:100A8200AD077FA012606F902802E0FEA3E078021B
:100A9200C333CE33CED8F92401FFE43EFE1260BD4B
:100AA200AD077FA112606F902802E0FEA3E07802FA
:100AB200C333CE33CED8F92402FFE43EFE1260BD2A
:100AC200AD077FA212606F902802E0FEA3E07802D9
:100AD200C333CE33CED8F92403FFE43EFE1260BD09
:100AE200AD077FA3803E7F91126062902895EFF060
:100AF2008035902895E0FD7FA080299027FFE0F4C3
:100B0200FD7FA012606F902800E0F4FD7FA11260CB
:100B12006F9027FFE004FD7F9112606F902800E044
:0F0B220004FD7F9212606F9027FDE0904000F07D
:010B310022A1
:104CE400904000E09027FDF0A37426F0A37488F0B0
:104CF4007BFF7A5279227D38FF7E261250C27D06D0
:104D0400E4FF12606F9027FEE0FEA3E07802CEC3BA
:104D140013CE13D8F9FD7FEC12606F9027FEE0FEEE
:104D2400A3E07802CEC313CE13D8F9EEFD7FED12C3
:104D3400606F9027FEE0FEA3E07802CEC313CE138B
:104D4400D8F9240DFD7FEE12606F9027FEE0FEA3DC
:104D5400E07802CEC313CE13D8F9240DE43EFD7FD0
:0C4D6400EF12606F9027FDE0904000F01F
:014D70002220
:104FE400902890E0FF6069904000E09027FDF0EF8A
:104FF40030E3107D0FE4FF12606F7B087D087F0BA8
:10500400125CC3E4FDFF12606F902890E030E00969
:105014007B027D027F31125CC3902890E030E1096D
:105024007B047D047F31125CC3902890E030E20958
:105034007B017D017F31125CC3902890E0FD7FA845
:1050440012606FE4902890F09027FDE0904000F00B
:015054002239
:10492400125E80902898EFF0125D8B125CE6120004
:104934000E7D09E4FF12606F7D017F6C12606FE4ED
:10494400FDFF12606F7D017F9E12606F7D877F9FE8
:1049540012606FE490288EF0A3F0902895F09028D0
:1049640092F0902890F090286A7420F09028EF74C8
:1049740001F0902903F09028C7E054FEF07D017FF8
:10498400AE12606F7D177FAF12606F90289CE0902D
:1049940028C77009E054FEF04402F08007E04401A7
:1049A400F054FDF09028C7E054DFF04440F0547F09
:1049B400F0E490286DF0125322122872125B6612F2
:0E49C4004CE41260EB125E44125C7B0256AFB4
:10548D00902891E060429028C2E06402703A902822
:10549D00C1E07034902896E0FEA3E0FF4E701090AE
:1054AD0028FBE0FDA3E0902896CDF0A3EDF022C3FC
:1054BD009028FCE09FFF9028FBE09EFED3EF94E840
:0954CD00EE940340031258612221
:103DD200902892E030E11F90288CE07002A3E070FE
:103DE200159028A1E0700F9028FBE0FFA3E0902837
:103DF2008CCFF0A3EFF090288CE0FEA3E0FF4E7092
:103E02001B9028A1E07015D39028FCE0949890288C
:103E1200FBE0940840069028A17401F09028A1E0EC
:103E22006003023EC9D3EF9400EE94005003023EB9
:013E3200C9C6
:103E330090288CE0FEA3E0FF9028FBE0FCA3E0FDCC
:103E4300D39FEC9E4006ED9FFFEC80139028FBE090
:103E5300FEA3E0FFC390288DE09FFF90288CE09E97
:103E63009027FDF0A3EFF0D39027FEE0940890276E
:103E7300FDE0940740509028A17401F0902891E050
:023E8300704489
:103E8500904000E09027FFF090289C7401F07D029F
:103E9500E4FF12606F7B087D087F12125CC37F0A06
:103EA5007E00125A587B08E4FD7F12125CC37F0A1C
:103EB5007E00125A589027FFE0FDE4FF12606F7EE6
:043EC500FF7FFF225A
:043EC900E4FEFF22F2
:1049D200E49027FDF09040007403F07F18126062AB
:1049E200EF54089027FDF070499028A1E0604390B1
:1049F20028F4E0FEA3E0FF4E70119028FBE0FDA337
:104A0200E09028F4CDF0A3EDF0803B9028F9E0701F
:104A120035C39028FCE09FFF9028FBE09EFED3EF79
:104A22009410EE9427401F1260479028F97401F009
:104A320080149028F9E0600E125E62E49028F9F08A
:104A42009028F4F0A3F09027FDE060119028F4E0A4
:104A52007002A3E06007E49028F4F0A3F09029022A
:104A6200E0601A902894E004F0E0D3946474809497
:0D4A720080400AE4FF1260B5E4902894F043
:014A7F002214
:0B55A600902840EBF0A3EAF0A3E9F02E
:1055B1009040007406F0E4FFEFC39D502390284013
:1055C100E0FBA3E0FAA3E0F98F82758300122412B5
:1055D100FE74C02FF582E4342EF583EEF00F80D8EF
:0955E1007B017D017FE7025CC340
:105825009040007406F0902EC0E09027FDF0902E79
:10583500C2E09027FEF09028CFE0245F600D047051
:10584500159027FDE0FF125B10800B9027FDE0FF10
:0B585500A3E0FD1256EFE49028D0F015
:015860002225
:10538100124924120632902895E020E003123CD6FF
:10539100902895E020E103125E26902895E020E216
:1053A100031239C6902895E020E703124FE4123D1D
:1053B100D2EF4E70CB902892E06002E4F09028D0BA
:1053C100E0600312582512548D1249D29028EDE065
:0F53D10060B1124C4F124BB8E49028EDF080A45D
:092B0E004228FB00004128FE00F2
:0D605500D288C289D2A8D28AC28BC2AA22E8
:105FC300E58954F04401F589758CFF758A9CD2A943
:035FD300D28C224B
:105A2700C2AC75C8347598505387BF4387407D68AB
:105A37007C00C3E49DE49CF5CBC3E49468F5CA8578
:105A4700CBCD85CACCE4902893F0902899F0D2ACBE
:015A5700222C
:105D8B00C2AF126055125FC3125A27E4904000F065
:0F5D9B0090401CF0A374DAF0A374FFF0D2AF2293
:03000300021D6576
:101D6500C0E0C083C082C0D075D000C000C001C033
:091D750002C004C005C006C0074D
:101D7E00904000E09027F5F0904000E4F090401085
:101D8E00E0FAA3E09027FAF0904012E09027FBF0E3
:101D9E00EA30E60E902892E04401F09028CBE04421
:101DAE0001F0EA30E30E902892E04402F09029040C
:101DBE00E04401F0EA30E40E902892E04404F09002
:101DCE002890E04480F0EA30E507902892E044083D
:101DDE00F09027FAE0FE20E004EA30E70E90289219
:101DEE00E04440F09028EEE04480F0EE30E50E90B6
:101DFE002892E04420F0902904E04402F090400044
:101E0E007406F09040F0E0FFA3E09027FCF09040C5
:101E1E00F2E0FE9027F7F09040F3E0FD9027F8F007
:101E2E009040F4E0FC9027F6F09040F5E09027F912
:101E3E00F0A904EFF58264406006E58264C0700E7E
:101E4E009028D07401F09027FCE09028CFF09028D5
:101E5E00A1E0702AEF546064207023EF541F6401D8
:101E6E00701C9027F6E070169027F9E0F582640357
:101E7E006006E582640570069028917401F0902842
:101E8E0090E030E7349040F5E0FFF582758300D3A3
:101E9E009400748094804021E5829405748094802F
:101EAE005017902890E0FCEF14FFF87401088002A0
:101EBE00C333D8FC4C902890F0EA30E2249027F7F8
:101ECE00E0FFD394007480948040169027F6E014BF
:101EDE00700F9028C8E054F04FF09028CBE04402E9
:101EEE00F0EA20E103021FF29040F5E09028CEF0D8
:101EFE0024FD602E24F8606314602224FD601424F7
:101F0E00FC607424FE601124106003021F9F902851
:101F1E00CB805E9028CB80679028CB80709028CBAA
:101F2E008041ED640170099028CCE04401F080619D
:101F3E00ED6402705CEE70099028CCE04402F080F3
:101F4E0050AF06D3EF9402748094809028CCE0506A
:101F5E00054404F0803B4408F08036ED64017009BE
:101F6E009028CCE04410F08028ED64027023902875
:101F7E00CCE04420F0801AED640170099028CCE08A
:101F8E004440F0800CED640270079028CCE0448051
:101F9E00F09027F8E0FD7C0064017014E964017094
:101FAE000F9028CE7405F09028CBE04420F08034BA
:101FBE00ED64014C7014E96482700F9028CE740F9A
:101FCE00F09028CBE04440F0801A9027F8E06401AE
:101FDE007012E96404700D9028CE7415F09028CB21
:101FEE00E04480F0904000E4F0904010EAF090273A
:101FFE00FAE0904011F09040ABE004F09040AAEA75
:10200E00F09027F5E0904000F0C2899028FEE004A1
:01201E00F0D1
:10201F00D007D006D005D004D002D001D000D0D048
:07202F00D082D083D0E03223
:0660D9009028FEE0FF220A
:03000B0002465D4D
:10465D00C0E0C0F0C083C082C0D075D000C000C023
:01466D000745
:10466E00758CFE758A0C90288EE475F0011224A9C3
:10467E00E5F020E0759028FCE004F070069028FB31
:10468E00E004F09028F1E004F0D394147480948048
:10469E00400B9028ED7401F09028F1E4F090289AE8
:1046AE00E07002A3E0600E90289BE024FFF09028BB
:1046BE009AE034FFF09028D1E0C394FF7480948088
:1046CE005003E004F09028D2E0C394FF74809480ED
:1046DE005003E004F0904000E0FFE4F090288EA339
:1046EE00E09040ACF0904000EFF0902872E0600255
:0246FE0014F0B6
:0F470000D007D000D0D0D082D083D0F0D0E0321C
:030023000260DF99
:0660DF00309802C2983265
:0D60620074002FF582E43440F583E0FF2246
:0D606F0074002FF582E43440F583EDF0223B
:105CC30074002FF582E43440F583E0FEEBF4FCEE40
:105CD3005CFEED5B4EFE74002FF582E43440F583E9
:025CE300EEF0E1
:015CE500229C
:0660BD008F828E83E0FFDC
:0160C30022BA
:0D607C00C3EE943050068F828E83EDF0222B
:1050C200902802EDF0A3EBF0A3EAF0A3E9F0902818
:0650D20000EEF0A3EFF078
:1050D800C3EE9430504EE4902806F0A3F0902802D6
:1050E800E0FF902806E0FCA3E0FDC39FEC9400508D
:1050F80033902803E0FBA3E0FAA3E0F98D828C83C8
:10510800122412FF902800E0FAA3E02DF582EA3C71
:10511800F583EFF0902807E004F070C1902806E0CE
:0451280004F080B956
:01512C002260
:0C609600902872EFF0902872E070FA225F
:105A880001B901E0037203C006E407800DC80F00E6
:105A98001B901E00014022223242C222223242C200
:0F5AA80022223242C23032383A3C3E3E3E3E3E2F
:102B17005A28C70000000000000000000000000065
:102B2700000000000000000000000000004B28B378
:102B37000203050608090B0C0E0F014828BF000009
:102B47000002ED0F00004228E26DB64128E5004182
:032B570028BEFF96
:10543E007D02E4FF12606F7F13126062EFC45403AB
:10544E0014601414600A14701A9027FE747F800C76
:10545E009027FE740F80059027FE7401F0A374FF51
:10546E00F080099027FEE4F0A3743FF09027FEE051
:0E547E00FEA3E0FF9028E2E05EF0A3E05FF006
:01548C0022FD
:10287200E49028D1F09028CAF09028C9F09028C896
:10288200F09028C7E0C3135401FF1245AA904000FC
:10289200E09027FDF07D07E4FF12606FE4FD7F0208
:1028A20012606FE4FD7F0112606F7D017F04126090
:1028B2006F7DFF7F0312606F7D507F0512606FE4B2
:1028C200FD7F0612606F7BF07D107F0A125CC37B76
:1028D200017D017F0A125CC37B037D017F50125C84
:1028E200C37B0F7D067F40125CC37D027F21126095
:1028F2006FE4FD7F2012606F7D037F2312606F7D86
:10290200FF7F2212606F7D037F2412606F7D067F3E
:102912000B12606F7D1A7F6512606F7D08E4FF12F3
:10292200606F7B407D407F10125CC37BC07DC07FA7
:1029320015125CC37B107D107F15125CC37B207D5A
:10294200207F0D125CC37D03E4FF12606F7B02E403
:10295200FD7F03125CC37B04E4FD7F01125CC37B39
:10296200E07D807F03125CC37B387D087F04125CAC
:10297200C37B10E4FD7F03125CC37B087D087F1ECE
:10298200125CC37BC0E4FD7F1E125CC37B08E4FDC6
:102992007F2A125CC37B307D207F2B125CC37B01BC
:1029A200E4FD7F03125CC37B807D807F2B125CC3BE
:1029B2007D967F1D12606F7D04E4FF12606F7B02C3
:1029C200E4FD7F03125CC37BE07D807F03125CC366
:1029D2007B387D087F04125CC37B087D087F1E1252
:1029E2005CC37BC0E4FD7F1E125CC37B807D807F65
:1029F2002B125CC37D967F1D12606F7D05E4FF1272
:102A0200606F7B087D087F0F125CC37D107F1712F9
:102A1200606F7B307D207F45125CC37D01E4FF1235
:102A2200606F7B077D027F01125CC37D8A7F091282
:102A3200606F7D02E4FF12606F7D077F1812606F86
:102A4200E4FD7F0112606FE4FD7F0212606FE4FD1E
:102A52007F0312606FE4FD7F0412606FE4FD7F0567
:102A620012606F7D407F0612606FE4FDFF12606F9F
:102A72007D207F0112606F7B047D047F30125CC376
:102A82007D06E4FF12606F7B01E4FD7F01125CC3EF
:102A92007D0FE4FF12606F7B037D027F2A125CC30D
:102AA2007B307D207F29125CC39027FDE09040009F
:102AB200F012543E120026123BD712441F7F01121D
:072AC2000FA27F010225CEE7
:020FA200AD0799
:100FA400E4902800F0A3F09027FEF0A3F09027FE31
:100FB400E0FEA3E0FFC3940FEE64809480503B7E78
:100FC400007401A807088005C333CE33CED8F9FFD7
:100FD400902804EEF0A3EFF09028E2E05EFEA3E098
:100FE4005F4E6006902800E004F09027FFE004F0D4
:100FF40070BB9027FEE004F080B3ED1470099028D4
:10100400027420F0A3E4F0E49027FEF0A3F090270C
:10101400FEE0FEA3E0FFC3940FEE648094804003DF
:101024000213647E007401A807088005C333CE331D
:10103400CED8F9FF902804EEF0A3EFF09028E2E078
:101044005EFEA3E05F4E70030213509027FEE0FEA5
:10105400A3E0FF7C007D03122473EC702DED14607B
:101064001314601C2402702290280612250200002A
:101074007D0080169028061225020000AC44800AE8
:101084009028061225020000BB80902806E0FCA3ED
:10109400E0FDA3E0FEA3E0FFC004C005C006C00756
:1010A4009027FEE0FEA3E0FF7C007D03122473A9D9
:1010B40007D007D006D005D004A8011224E3902855
:1010C400061224F6902801E060030211AAA375F029
:1010D400011224A9AFF0FEC006C007902806E0FC68
:1010E400A3A3A3E0FFE4AD07D007D00612607C9071
:1010F4002802E475F0011224A9AFF0FEC006C0076F
:10110400902806E0FCA3E0FDA3E0FEA3E0FF78083E
:101114001224D0E4AD07D007D00612607C902802D8
:10112400E475F0011224A9AFF0FEC006C0079028B0
:1011340006E0FCA3E0FDA3E0FEA3E0FF7810122488
:10114400D0E4AD07D007D00612607C902802E47585
:10115400F0011224A9AFF0FEC006C007902806E0F3
:10116400FCA3E0FDA3E0FEA3E0FF78181224D0E482
:10117400AD07D007D00612607C902802E475F00118
:101184001224A9AFF0FE902800E0FD12607C9028A4
:1011940002E475F0011224A9AFF0FEE4FD12607CB4
:1011A4009028017401F0902802E475F0011224A93A
:1011B400AFF0FEC006C007902806E0FCA3A3A3E09E
:1011C400FFE4AD07D007D00612607C902802E475D6
:1011D400F0011224A9AFF0FEC006C007902806E073
:1011E400FCA3E0FDA3E0FEA3E0FF78081224D0E412
:1011F400AD07D007D00612607C902802E475F00198
:101204001224A9AFF0FEC006C007902806E0FCA394
:10121400E0FDA3E0FEA3E0FF78101224D0E4AD07C4
:10122400D007D00612607C902802E475F0011224E5
:10123400A9AFF0FEC006C007902806E0FCA3E0FDBD
:10124400A3E0FEA3E0FF78181224D0E4AD07D00792
:10125400D00612607C902802E475F0011224A9AF34
:10126400F0FEC006C007902806E0FCA3A3A3E0FF9D
:10127400E4AD07D007D00612607C902802E475F034
:10128400011224A9AFF0FEC006C007902806E0FCB6
:10129400A3E0FDA3E0FEA3E0FF78081224D0E4ADB0
:1012A40007D007D00612607C902802E475F0011282
:1012B40024A9AFF0FEC006C007902806E0FCA3E016
:1012C400FDA3E0FEA3E0FF78101224D0E4AD07D024
:1012D40007D00612607C902802E475F0011224A95C
:1012E400AFF0FEC006C007902806E0FCA3E0FDA313
:1012F400E0FEA3E0FF78181224D0E4AD07D007D0B5
:101304000612607C902802E475F0011224A9AFF063
:10131400FEE4FD12607C902802E475F0011224A919
:10132400AFF0FEE4FD12607C902802E475F0011237
:1013340024A9AFF0FEE4FD12607C902802E475F06D
:10134400011224A9AFF0FEE4FD12607C9027FFE0B7
:1013540004F060030210129027FEE004F002101261
:011364002266
:1025CE00902802E4F0A304F0902808E4F0A37480AD
:1025DE00F090280474C0F0A37480F0E4A3F0A3F08C
:1025EE00EF1470109028007421F0A374C4F090279B
:1025FE00FE7402F0E49027FFF09027FEE0FFA3E0C8
:10260E00D39F40030228719028C7E090280020E055
:10261E000302272FE475F0011224A9AFF0FEE4FDAA
:10262E0012607C902800E475F0011224A9AFF0FE30
:10263E00E4FD12607C902800E475F0011224A9AF2D
:10264E00F0FEE4FD12607C902800E475F001122487
:10265E00A9AFF0FEE4FD12607C902800E475F00155
:10266E001224A9AFF0FE902804A3E0FD12607C9026
:10267E002800E475F0011224A9AFF0FE902804E0C2
:10268E00FD12607C902800E475F0011224A9AFF0D1
:10269E00FEE4FD12607C902800E475F0011224A97E
:1026AE00AFF0FEE4FD12607C902800E475F001129C
:1026BE0024A9AFF0FE902806A3E0FD12607C9028BE
:1026CE0000E475F0011224A9AFF0FE902806E0FD9B
:1026DE0012607C902800E475F0011224A9AFF0FE80
:1026EE00E4FD12607C902800E475F0011224A9AF7D
:1026FE00F0FEE4FD12607C902800E475F0011224D7
:10270E00A9AFF0FE902808A3E0FD12607C9028008F
:10271E00E475F0011224A9AFF0FE902808E002281B
:10272E0040E475F0011224A9AFF0FEE4FD12607CC6
:10273E00902800E475F0011224A9AFF0FEE4FD121A
:10274E00607C902800E475F0011224A9AFF0FEE43D
:10275E00FD12607C902800E475F0011224A9AFF000
:10276E00FEE4FD12607C902800E475F0011224A9AD
:10277E00AFF0FE902802A3E0FD12607C902800E4EA
:10278E0075F0011224A9AFF0FE902802E0FD126050
:10279E007C902800E475F0011224A9AFF0FE902879
:1027AE0004A3E0FD12607C902800E475F001122471
:1027BE00A9AFF0FE902804E0FD12607C902800E4A2
:1027CE0075F0011224A9AFF0FE902806A3E0FD12C9
:1027DE00607C902800E475F0011224A9AFF0FE9001
:1027EE002806E0FD12607C902800E475F0011224AA
:1027FE00A9AFF0FE902808A3E0FD12607C9028009F
:10280E00E475F0011224A9AFF0FE902808E0FD1245
:10281E00607C902800E475F0011224A9AFF0FEE46C
:10282E00FD12607C902800E475F0011224A9AFF02F
:10283E00FEE4FD12607C902800E475F0011224A9DC
:10284E00AFF0FEE4FD12607C902800E475F00112FA
:10285E0024A9AFF0FEE4FD12607C9027FFE004F0A7
:03286E0002260738
:012871002244
:100026007D06E4FF12606F9028C7E030E00302050A
:100036006C9027FE743CF0A37408F0A3E4F09027BC
:10004600FFA3E0FD7F3C12606F9027FEE004FFA354
:10005600E0FD12606F9027FEE004FF7BF07D7012DA
:100066005CC39027FEE02402FF7D0512606F902797
:10007600FEE02403FF7D0112606F9027FEE024045A
:10008600FFE4FD12606F9027FEE02405FF7D10124D
:10009600606F9027FEE02406F0A37408F0A37401B5
:1000A600F09027FEE0FFA3A3E0FD12606F9027FE0D
:1000B600E004FFA3E0FD12606F9027FEE004FF7BE3
:1000C600F07DB0125CC39027FEE02402FF7D05128E
:1000D600606F9027FEE02403FF7D0112606F90277A
:1000E600FEE02404FFE4FD12606F9027FEE0240585
:1000F600FF7D1012606F9027FEE02406F0A37408BF
:10010600F0A37420F09027FEE0FFA3A3E0FD1260A9
:100116006F9027FEE004FFA3E0FD12606F9027FEBC
:10012600E004FF7BF07D70125CC39027FEE02402A2
:10013600FF7D0F12606F9027FEE02403FF7D011202
:10014600606F9027FEE02404FFE4FD12606F9027A5
:10015600FEE02405FF7D1012606F9027FEE0240666
:10016600F0A37408F0A37421F09027FEE0FFA3A388
:10017600E0FD12606F9027FEE004FFA3E0FD126031
:100186006F9027FEE004FF7BF07DB0125CC39027E2
:10019600FEE02402FF7D0F12606F9027FEE024032D
:1001A600FF7D0112606F9027FEE02404FFE4FD123C
:1001B600606F9027FEE02405FF7D1012606F902788
:1001C600FEE02406F0A37408F0A37460F09027FE06
:1001D600E0FFA3A3E0FD12606F9027FEE004FFA3FB
:1001E600E0FD12606F9027FEE004FF7BF07D501269
:1001F6005CC39027FEE02402FF7D0512606F902706
:10020600FEE02403FF7D0212606F9027FEE02404C7
:10021600FFE4FD12606F9027FEE02405FF7D1012BB
:10022600606F9027FFE0FEA3E07802C333CE33CEA3
:10023600D8F9FF7D0112607C9027FEE02406F0A32A
:100246007408F0A37464F09027FEE0FFA3A3E0FD1A
:1002560012606F9027FEE004FFA3E0FD12606F902E
:1002660027FEE004FF7BF07D50125CC39027FEE082
:100276002402FF7D0F12606F9027FEE02403FF7DAE
:100286000212606F9027FEE02404FFE4FD12606F07
:100296009027FEE02405FF7D1012606F9027FFE097
:1002A600FEA3E07802C333CE33CED8F9FF7D011228
:1002B600607CE4902801F0A3F0FDEDD394047480F3
:1002C6009480501E7E007401A805088005C333CEB5
:1002D60033CED8F9FF902801E04EF0A3E04FF00DA1
:1002E60080D89027FEE02406F0A37408F0A374617A
:1002F600F09027FEE0FFA3A3E0FD12606F9027FEBB
:10030600E004FFA3E0FD12606F9027FEE004FF7B90
:10031600F07D50125CC39027FEE02402FFE4FD123C
:10032600606F9027FEE02403FF7D0212606F902726
:10033600FEE02404FFE4FD12606F9027FEE0240532
:10034600FF7D1112606F9027FFE0FEA3E07802C3E5
:1003560033CE33CED8F9FF7D0212607C9027FFE0C2
:10036600FEA3E07802C333CE33CED8F92401FFE4EE
:100376003EFE902801A3E0FD12607C9027FFE0FE80
:10038600A3E07802C333CE33CED8F92402FFE43E8D
:10039600FE902801E0FD12607C9027FFE0FEA3E0BE
:1003A6007802C333CE33CED8F92403FFE43EFEE40D
:1003B600FD12607C9027FFE0FEA3E07802C333CEF7
:1003C60033CED8F92404FFE43EFEE4FD12607CE45B
:1003D600902801F0A3F0FDEDD3940474809480502E
:1003E6001E7E007401A805088005C333CE33CED81F
:1003F600F9FF902801E04EF0A3E04FF00D80D89071
:1004060027FEE02406F0A37408F0A37465F0902795
:10041600FEE0FFA3A3E0FD12606F9027FEE004FF5D
:10042600A3E0FD12606F9027FEE004FF7BF07D5095
:10043600125CC39027FEE02402FFE4FD12606F9079
:1004460027FEE02403FF7D0212606F9027FEE02462
:1004560004FFE4FD12606F9027FEE02405FF7D1285
:1004660012606F9027FFE0FEA3E07802C333CE331D
:10047600CED8F9FF7D0212607C9027FFE0FEA3E054
:100486007802C333CE33CED8F92401FFE43EFE9082
:100496002801A3E0FD12607C9027FFE0FEA3E07830
:1004A60002C333CE33CED8F92402FFE43EFE9028B1
:1004B60001E0FD12607C9027FFE0FEA3E07802C316
:1004C60033CE33CED8F92403FFE43EFEE4FD1260BA
:1004D6007C9027FFE0FEA3E07802C333CE33CED86C
:1004E600F92404FFE43EFEE4FD12607C9027FEE062
:1004F6002406F0A37408F0A37467F09027FEE0FFCB
:10050600A3A3E0FD12606F9027FEE004FFA3E0FDC9
:1005160012606F9027FEE004FF7BF07D70125CC3D3
:100526009027FEE02402FF7D0C12606F9027FEE00C
:100536002403FF7D0112606F9027FEE02404FFE490
:10054600FD12606F9027FEE02405FF7D1012606F9C
:100556009027FFE0FEA3E07802C333CE33CED8F96E
:10056600FFE4FD02607C9027FE743CF0A37408F063
:10057600A3E4F09027FFA3E0FD7F3C12606F902775
:10058600FEE004FFA3E0FD12606F9027FEE004FF8B
:100596007BF07D70125CC39027FEE02402FFE4FD31
:1005A60012606F9027FEE02403FF7D0112606F90BA
:1005B60027FEE02404FFE4FD12606F9027FEE0248E
:1005C60005FF7D2112606F9027FEE02406F0A374DC
:1005D60008F0A37420F09027FEE0FFA3A3E0FD122D
:1005E600606F9027FEE004FFA3E0FD12606F902786
:1005F600FEE004FF7BF07D70125CC39027FEE024D2
:1006060002FFE4FD12606F9027FEE02403FF7D01E8
:1006160012606F9027FEE02404FFE4FD12606F90E5
:0B06260027FEE02405FF7D2212606F1C
:0106310022A6
:103BD7009027FE74A8F0A37408F0A37470F07D0614
:103BE700E4FF12606F9027FEE0FFA3A3E0FD1260E1
:103BF7006F9027FEE004FFA3E0FD12606F9027FEA1
:103C0700E02402FF7D0312606F9027FEE02403FF8C
:103C17007D0112606F9027FEE02404FFE4FD12602F
:103C27006F9027FEE02405FF7D0112606F9027FE4D
:103C3700E02406FFE4FD12606F9027FFE0FEA3E09B
:103C47007802C333CE33CED8F9FFE4FD12607C90FF
:103C570027FEE02407F0A37408F0A37480F07D0624
:103C6700E4FF12606F9027FEE0FFA3A3E0FD126060
:103C77006F9027FEE004FFA3E0FD12606F9027FE20
:103C8700E02402FF7D0B12606F9027FEE02403FF04
:103C97007D0112606F9027FEE02404FFE4FD1260AF
:103CA7006F9027FEE02405FF7D0112606F9027FECD
:103CB700E02406FFE4FD12606F9027FFE0FEA3E01B
:0F3CC7007802C333CE33CED8F9FFE4FD02607C20
:10441F007D06E4FF12606F9027FE74C4F0A374084A
:10442F00F0A37471F09027FFA3E0FD7FC412606FBB
:10443F009027FEE004FFA3E0FD12606F9027FEE0DF
:10444F002402FF7D0312606F9027FEE02403FF7D9F
:10445F00FF12606F9027FEE02404FF7D0112606F52
:10446F009027FEE02405FF7DFF12606F9027FEE08E
:10447F002406FF7D0112606F9027FEE02407F0A352
:10448F007408F0A37481F09027FEE0FFA3A3E0FD72
:10449F0012606F9027FEE004FFA3E0FD12606F90A3
:1044AF0027FEE02402FF7D0B12606F9027FEE024B1
:1044BF0003FF7DFF12606F9027FEE02404FF7D0154
:1044CF0012606F9027FEE02405FF7DFF12606F9052
:0B44DF0027FEE02406FF7D0102606F55
:1059BC00D3EF9400EE9480E4401D9FFFE49EFE74B0
:1059CC00019400FDE49400FC78011224E390280B70
:1059DC00EEF0A3EFF0800690280BF0A3F090280BCC
:0559EC00E0FEA3E0FF56
:0159F1002293
:06470F009028041224F6BC
:10471500E4902808F0902808E0FFC3940A74809478
:10472500805062EF30E009E47F807EBBFDFC8007AE
:10473500E47F447EACFDFC9028091224F6902809FC
:10474500E0FCA3E0FDA3E0FEA3E0FF902808E0FB6A
:10475500C313F9F81224E3A31224F6902809E0FC08
:10476500A3E0FDA3E0FEA3E0FF902804E0F8A3E0AA
:10477500F9A3E0FAA3E0FBC31224BF600890280860
:10478500E004F08090902808E0C3940A7480948037
:104795004024E4FF7E7DFDFC902804E0F8A3E0F9C9
:1047A500A3E0FAA3E0FB1224BF70047F0A80027F16
:0B47B50001902808EFF0902808E0FFBA
:0147C00022D6
:05487300902800EFF0A9
:10487800E4FF126062902802EFF0902800E024F034
:10488800603A14606124F160292420600302491A07
:104898009021C0E0902801F0E05401C454F0FE904B
:1048A80028DBE054EFFCA3E0FDEC4EFFED9028DBA5
:1048B800802A902200E0902801F08056902240E063
:1048C800902801F0E05401C454F0FE9028DDE05433
:1048D800EFFCA3E0FDEC4EFFED9028DDCFF0A3EF59
:1048E800F0E4FDFF8029902240E0902801F0E05498
:1048F80001C454F0FE9028DDE054EFFCA3E0FDEC89
:104908004EFFED9028DDCFF0A3EFF0E4FD7F01121C
:0C491800427D902802E0FDE4FF02606F89
:10591400EF14702CED75F010A424C5F582742135B4
:10592400F0F583E0FAED75F010A424C4F582742137
:1059340035F0F583E0FFEAFE902808EEF0A3EFF0DF
:08594400902808E0FEA3E0FF3B
:01594C002238
:053FC100902800EFF064
:103FC600ED54F024F0600F24F060162420701D904C
:103FD6002803740180109028037401F0A304F08074
:103FE6000B9028037403F0ED540FA3F0E4FF126066
:0F3FF60062902801EFF0902800E0600302409FE6
:104005009021C5E0FE9021C4E0FDEDFF1259BCAB47
:1040150007AA069021D5E0FE9021D4E0FDEDFF1220
:1040250059BC902805EEF0A3EFF09021E5E0FE9055
:1040350021E4E0FDEDFF902809EEF0A3EFF09028D4
:1040450009E0FEA3E0FF1259BC902807EEF0A3EFAC
:10405500F0E4902802F0902806E02B902805E03A3D
:104065009028FFF0AE02AF03902808E02F902807B4
:10407500E03E902900F0D39028C0E0940A9028BF34
:10408500E09400400A1247C1E49028BFF0A3F090E5
:0A40950028FFE0FFA3E0FD1260E841
:0A409F00902801E0FDE4FF02606FCD
:1055EA00EF24F4703590219CE09027FDF0E4FF123F
:1055FA0060629027FEEFF07D05E4FF12606F90274E
:10560A00FDE0640170047F0180027F00EF333333D1
:10561A0054F8FD7B087F0F125CC39027FEE0FDE47F
:04562A00FF02606FAC
:105C5600904000E09027FDF0E4FDFF12606F7F3278
:105C66001260629027FDE0904000F0EF30E4037F81
:045C760001227F0088
:015C7A002207
:0545AA009027FEEFF078
:1045AF00904000E09027FFF09028C7E0FF30E00434
:1045BF007E0A80027E50902800EEF09027FEE06485
:1045CF00017008EF30E0047F0780027F0090280120
:1045DF00EFF07D08E4FF12606F902800E0FD7F028E
:1045EF0012606F7D07E4FF12606F902801E0FFC437
:1045FF0054F0FEEF4EFD7F0E12606F9027FEE070BD
:10460F00047D0380027D067B0F7F40125CC37D0A11
:10461F00E4FF12606F902800E0FD7F0212606F7D53
:10462F0009E4FF12606F902801E0FD7B0F7F0E12EF
:10463F005CC39027FEE070047D0380027D067B0F34
:0D464F007F40125CC39027FFE0904000F018
:01465C00223B
:05363B00902804EDF0F1
:10364000904000E0902805F0EF24F060072410601F
:10365000030237697D08E4FF12606F902804E0FFE1
:10366000C3940A74809480503DEF30E009E4FFFE7B
:103670007DE07C2E80087F787E397D057C33902824
:10368000071224F6902807E0FCA3E0FDA3E0FEA3C8
:10369000E0FF902804E0FBC313F9F81224D090282F
:1036A000071224F6800A90280712250246500000CF
:1036B000E4902806F0902806E0FFC39404748094F8
:1036C000805039EF2408FFC007A3E0FCA3A3E0FE6D
:1036D000A3E0FFE4AD07D00712606F902807E0FC7D
:1036E000A3E0FDA3E0FEA3E0FF78081224D0902819
:1036F000071224F6902806E004F080B9902804E030
:1037000025E02488F582E4345AF583E4740193FDBE
:103710007F0612606F902804E025E02488F582E49B
:10372000345AF583E493FD7F0712606F9028D6E04A
:10373000C4540FFF902804E06F60197B807D807F68
:103740000C125CC3902804E0C454F0FF9028D6E02B
:10375000540F4FF07D03E4FF12606F902804E09057
:103760005AAD93FD7F2712606F902805E0904000CE
:01377000F068
:013771002235
:0B38A500902804EFF0A3EDF0A3EBF07F
:1038B000904000E0902807F07D07E4FF12606F7DE4
:1038C000027F0512606F902806E0C454F0FD7BF083
:1038D0007F0A125CC3902806E0C454F0FD7BF07FA1
:1038E00040125CC3E4FD7F0212606FE4FD7F0112B1
:1038F000606F902804E0131313541FFFC374049FD8
:10390000FD7B037F07125CC3902805E0C454F0FDE3
:103910007BF07F07125CC3902805E064067003FF0C
:1039200080027F01EF146019146016240270249045
:10393000280B7401F0A374F8F09028087423F08029
:103940002190280B7401F0A374F8F09028087417E4
:10395000F0800F90280B7402F0A3E4F09028087414
:103960001FF090280CE024FFFE90280BE034FF901D
:103970002809F0A3CEF0902809E0FD7F0412606FC3
:10398000902809A3E0FD7F0312606F902808E0FDF6
:103990007B3F7F08125CC39028C7E030E0047D5075
:1039A00080027D0A7F0512606F7D03E4FF12606F65
:1039B000902805E014FD7B077F1E125CC39028074A
:0539C000E0904000F062
:0139C50022DF
:104A8000904000E0902802F0EF75F003A424D6F5E2
:104A900082E43428F583E054F0902803F0EF7004AA
:104AA0007D0380027D04E4FF12606F902803E0FF25
:104AB000C0077F03126062EF30E4047E0880027E4C
:104AC00000D0E04E902803F0E0FFC0077F051260A1
:104AD00062EF30E6047E0480027E00D0E04E902833
:104AE00003F0E0FFC0077F18126062EF30E1047E40
:104AF0000280027E00D0E04E902803F0E0FFC00765
:104B00007F18126062EF30E3047E0180027E00D0E5
:0F4B1000E04EFF902803F0902802E0904000F064
:014B1F002273
:074276009027FDE0FF7D0130
:0A427D00902806EDF0902805EFF000
:10428700904000E0902807F0EF70297D03FF12604F
:104297006F9028C7E01313543F30E0059028DD8066
:1042A700039028DBE0C4540F7E005401FF902808D8
:1042B700EFF080127D04E4FF12606F9028DDE0C408
:1042C7005401902808F0902806E020E0069028087E
:1042D700E060357B017D017F01125CC37B087D08AF
:1042E7007F1E125CC37B807D807F21125CC37F01B0
:1042F7001260B5902805E090286D7006E04404F040
:104307008039E04410F080337B01E4FD7F01125CCB
:10431700C37B08E4FD7F1E125CC37B80E4FD7F2125
:10432700125CC3902805E090286D7006E054FBF0FE
:104337008004E054EFF0E4FF1260B5902807E090A6
:034347004000F043
:01434A002250
:08598500902802EEF0A3EFF000
:10598D00904000E0902804F07D03E4FF12606F90DA
:10599D002802E07002A3E060047D0280027D007B9E
:0E59AD00027F03125CC3902804E0904000F0DB
:0159BB0022C9
:0A40A900902803EDF0902802EFF0DC
:1040B300904000E0902804F0EF70047D0380027DBF
:1040C30004E4FF12606F902803E024E0602F24F0E3
:1040D3006052242070787BC0E4FD7F05125CC37BB3
:1040E30010E4FD7F03125CC3902802E070047D0797
:1040F30080027D09E4FF12606F7D50804C7BC0E439
:10410300FD7F05125CC37B107D107F03125CC3909F
:104113002802E070047D0780027D09E4FF12606FCE
:104123007D0A80257BC07DC07F05125CC37B107D2B
:10413300107F03125CC3902802E070047D078002A5
:104143007D09E4FF12606F7D0A7F0512606F90287E
:1041530004E0904000F0902802E0FFA3E0FD12424B
:104163007D902803E030E413902802E090286D70DE
:1041730005E04402F022E04408F022902802E09097
:0D418300286D7005E054FDF022E054F7F0C7
:01419000220C
:050B32009027FDEFF02B
:100B3700124A80902800EFF09027FDE0FF75F00340
:100B4700A424D5F582E43428F583E0FE9027FFF04E
:100B57009027FEF0EF75F003A424D7F582E434283C
:100B6700F583E0902801F09028BEE06E602A902778
:100B7700FEE09028BEF024FD601424DE600824F017
:100B870060042420700D9028E17401F08005E49042
:100B970028E1F0E49028E4F09027FEE01225330BDB
:100BA700F2000BF7010C00020C09030C6A110C8A06
:100BB700130CD1140D55150DB5160E07170F171871
:100BC7000D01240D85250DDE260E2B270F20280E5F
:100BD70057310E64330E7D340ED0350EF3360F29A0
:100BE700380F32480F4E4A00000F4E1242768000EF
:100BF7009027FF7403F0020F541242769027FF7478
:100C070003F0902800E020E003020F549028F9E059
:100C1700600E125E62E49028F9F09028F4F0A3F0D9
:100C2700902801E0640160079028DBE030E60F9030
:100C370028DBE04440F09027FF7434F080129028BE
:100C4700C7E09027FF30E6057413F080037414F0B3
:100C5700E4902801F09028D1F09028DBE054DFF0F1
:100C6700020F54902800E020E003020F549028C799
:100C7700E09027FF30E6067413F0020EEC7414F0D0
:100C8700020EEC902800E0FFC4540FD39403748045
:100C970094805003020E119028D1E0D3946474809D
:100CA7009480400DEF9027FF30E103020E38020ECB
:100CB70051902801E0700A902800E030E003020F0D
:100CC700549027FF7402F0020F549028C8E0C454D0
:100CD7000FFF125FD69028C8E0C4540FC39408745E
:100CE7008094809027FDE0FF50087D101240A902F4
:100CF7000DBC7D011240A9020F549028C7E030E6D1
:100D070040A3E0C4540F24FCFFE434FFC313EF13E4
:100D1700FF125FE89028C8E0C4540F24FCFFE434B6
:100D2700FFFE7C007D02122473C3EF9403EE648000
:100D370094809027FDE0FF50047D20800B7D01808B
:100D4700079027FDE0FF7D011240A9020DE59028DD
:100D570001E0707A9028DBE030E50280719028008E
:100D6700E0FF30E1099027FF7418F0020EECEF3036
:100D7700E003020F549027FF7418F0020EEC90283E
:100D870001E070739028DBE030E502806A9028006C
:100D9700E0FF20E1099027FF7428F0020EECEF3006
:100DA700E003020F549027FF7428F0020EEC9028FE
:100DB70000E030E0099027FF7415F0020F549028E7
:100DC700D1E0D3940A748094805003020F54902783
:100DD700FF7418F0020F54902800E030E0099027C4
:100DE700FF7425F0020F549028D1E0D3940174804A
:100DF70094805003020F549027FF7428F0020F5479
:100E0700124276902800E020E1059027FF803B9072
:100E170028D1E0D39414748094805003020F549027
:100E270027FF800D124276902800E030E1099027D5
:100E3700FF7424F0020F549028D1E0D39478748083
:100E470094805003020F549027FF7414F0020F543C
:100E5700902800E030E0069027FF7434F09028D106
:100E6700E0D39414748094805003020F549027FFAA
:100E77007434F0020F549028C7E030E640A3E0C472
:100E8700540F24FEFFE434FFC313EF13FF125FFA7E
:100E97009028C8E0C4540F24FEFFE434FFFE7C0012
:100EA7007D02122473C3EF9403EE6480948090272D
:100EB700FDE0FF50047D30800B7D0180079027FD0A
:100EC700E0FF7D011240A9802A902801E070399047
:100ED70028DBE030E5028030902800E020E06E90CB
:100EE70027FF7438F0E49028D1F08061902800E063
:100EF70030E0089027FF7435F080529028D1E0D376
:100F070094147480948040459027FF7438F0803D96
:100F17009027FDE0FF7D1180199027FDE0FF7D21DF
:100F270080109027FDE0FF7D3180079027FDE0FFCF
:100F37007D8512427DE4FFFE125985E49028D1F0A9
:100F47009027FF04F080069027FF7401F090280097
:100F5700E0FF9027FDE0FE75F003A424D6F582E4B8
:100F67003428F583EFF0902801E0FFEE75F003A435
:100F770024D7F582E43428F583EFF09027FFE0FFCC
:100F87009027FEE06F60139027FDE075F003A4241F
:0A0F9700D5F582E43428F583EFF06D
:010FA100222D
:105F2600125C56EF540125E0FF9028C7E054FD4F60
:0A5F3600F0E0C3135401FF0245AA76
:0534F7009027FDEFF03D
:1034FC0014600302358E9028C8E0540F9027FEF01C
:10350C00902002E0FFE4FCFDFE78101224E3C004DE
:10351C00C005C006C007A3E0FFE4FCFDFE7818124E
:10352C0024E3D003D002D001D000EF4BFFEE4AFED3
:10353C00ED49FDEC48FCC004C005C006C007902056
:10354C0001E0FFE4FCFDFE78081224E3D003D00276
:10355C00D001D000EF4BFBEE4AFAED49F9EC48F8FC
:10356C00902000E0FFEB4FFFEAFEE9FDE8FC12477C
:10357C000F9027FFEFF09027FEE0905A9E93902833
:10358C0003F0902803E0FE540F902801F0EE5470E5
:10359C00C313902800F0902803E05480C413131335
:1035AC005401902802F09028C7E0FF30E00D9028DD
:1035BC0000E06420700F7410F0800AEF30E5069084
:1035CC0028007420F09027FDE01470629028C7E06A
:1035DC0020E24A7D01E4FF12427D9027FFE0FDE4EA
:1035EC00FF12363B902800E0FFA3E0FD7B01123870
:1035FC00A590286EE054FCFFF0902800E0C4540F16
:10360C00F04F90286EF09028DBE04420F054BFF08F
:10361C00902802E060079028DBE04440F09027FF00
:0E362C00E0C454F0FF9027FEE04F9028C8F055
:01363A00226D
:0C6089009028CEE0FF24F470031255EACA
:0160950022E8
:104191009027FF7402F0EF24FE605C24FE6075241A
:1041A100FC700302423424F8603524F0603124E0CD
:1041B100602F24C0700302425D247F6003024275B8
:1041C1009027FD7403F09028C8E0540F9027FEF06B
:1041D100E0905A9E93540F9027FFF0E4FF801580E2
:1041E100749027FD7413F09028C7E030E2047F102B
:1041F10080027F110248739027FD7403F09028C854
:10420100E0540F9027FEF0E0905A9E93540F9027B0
:10421100FFF0803C9027FD7403F09028C8E0540F14
:104221009027FEF0E0905A9E93540F9027FFF044A0
:1042310010801D9027FD7403F09028C8E0540F9062
:1042410027FEF0E0905A9E93540F9027FFF04420F0
:10425100FDE4FF801C9027FD740BF0229027FD7474
:1042610013F09028C7E07D0230E2047F1080027FC6
:0442710011123FC126
:014275002226
:10586100E49028C104F09021C5E0FE9021C4E0FD40
:10587100EEFC9021D5E0FE9021D4E0FBEB2DFDEE76
:105881003CAF059028C5F0A3EFF0E49028BFF0A34A
:0B589100F09028EE7402F09028F0F078
:01589C0022E9
:1047C1009021C5E0FE9021C4E0FDEDFF90280BEEA5
:1047D100F0A3EFF09021D5E0FE9021D4E0FDEDFFB4
:1047E10090280CE02FF090280BE03EF09028C5E0D7
:1047F100FEA3E0FF90280BE0B50627A3E0B5072252
:10480100E49028C1F09028FFE0FFA3E0FD125D2AAB
:104811009028EE7402F09028F014F09028C2E01471
:10482100F02290280BE0FEA3E0FF9028C5EEF0A354
:10483100EFF09028C3E0FCA3E0FDD3EF9DEE9C4098
:104841000B9028EE7402F09028F0F022E49028C139
:10485100F0A3F0A3E0FEA3E0FFC390280CE09F903B
:10486100280BE09E500B9028EE7402F09028F01473
:01487100F056
:014872002223
:10526200904000E09027FDF07D0BE4FF12606F7D1F
:10527200567F0112606F7B017D017F02125CC37D4C
:10528200097F0512606F7DA07F0412606FE4FFEF5B
:10529200C3940874809480500F74802FF582E43494
:1052A20026F583E4F00F80E77D027F0312606F7DB5
:1052B200087F0612606F9027FDE0FDE4FF02606F39
:105C0800904000E0902801F0902680EFF07D0BE4B2
:105C1800FF12606F7B017D017F07125CC390280132
:075C2800E0FDE4FF02606FE4
:1058D900904000E0902801F07D0BE4FF12606F7F9B
:1058E90008126062EF30E0167B01E4FD7F08125C6C
:1058F900C3902801E0FDE4FF12606F7F0122902828
:0A59090001E0FDE4FF12606F7F0073
:015913002271
:01000A0022D3
:0160F4002289
:0160F5002288
:0160F6002287
:104B2000902680E0FF902801F0902681E0FE9028FA
:104B300002F0902682E0902803F0902683E0FDA307
:104B4000E0FCA3E0902804F0902686E0F9EEFBEF6D
:104B50002BFFE433FE902682E07A002FFFEA3EFE30
:104B6000A3E02FFFEA3EFEA3E02FFFEA3EFEA3E014
:104B70002FFFEA3EFEEF69703E902680E064C7702A
:104B800036A3E064A57030902803E024FE60111481
:104B900060151460192403701EAF05AD0402000AED
:104BA000AF05AD040260F4AF05AD040260F5AF05DA
:074BB000AE04AD061260F631
:014BB70022DB
:101A1D0048494420496E7465726661636500694189
:101A2D005020496E74657266616365001201000293
:101A3D00EF020140C62F11600101010203011201E5
:101A4D000002EF020140C62F82F0010201020301E4
:101A5D0004030904050C0901A1011500250109E97B
:101A6D0009EA09E209B709CD09B509B6750195105D
:101A7D008102C0092111010001221F000A06000286
:101A8D00EF02014001000902C40003010080640956
:101A9D0004000000010100000924010001280001DB
:101AAD00010C24020101010002030000000A2406BA
:101ABD0003010103020200092403040103000300D2
:101ACD0009040100000102000409040101010102E1
:101ADD00000007240101010100142402010202107B
:101AED000444AC0080BB0088580100770109050152
:101AFD000D46020400000725010100010009040143
:101B0D000201010200000724010101010014240259
:101B1D00010203180444AC0080BB00885801007713
:101B2D00010905010D460204000007250101000110
:101B3D000009040200010300000709211101000141
:101B4D00221F000705860308000A09025001030140
:101B5D00008032080B000201002000090400000083
:101B6D000101200209240100020440000008240A9A
:101B7D000503070000112402010101000502030005
:101B8D000000000000001224060301030000000CF9
:101B9D000000000C000000000C24030401030003EE
:101BAD0005000000090401000001022004090401E0
:101BBD0001020102200010240101050101000000B5
:101BCD0002030000000006240201021007050105B2
:101BDD00080301082501000000000007058111041C
:101BED000004090401020201022000102401010574
:101BFD0001010000000203000000000624020103A1
:101C0D001807050105080301082501000000000063
:101C1D0007058111040004090401030201022000DB
:101C2D001024010105010100000002030000000065
:101C3D0006240201042007050105080301082501FA
:101C4D0000000000000705811104000409040104CF
:101C5D000201022000102401010501000000800294
:101C6D0003000000000624020104200705010508F9
:101C7D000301082501000000000007058111040083
:101C8D0004090402000103000007092111010001EC
:101C9D00221F000705860308000A0907BE0002017E
:101CAD0000C0000904000000010100000A24010029
:101CBD00013E000201020C24020101010002030099
:101CCD0000000A2406030101030202000924030493
:101CDD0001030003000C24020A03060002030000A6
:101CED00000924030D0101000A000904010000018F
:101CFD000200040904010101010200000724010191
:101D0D000101000E2402010202100244AC0080BB4E
:101D1D000009050109F0000100000725010100017E
:101D2D00000904020000010200050904020101017D
:101D3D000200000724010D0101000E240201020220
:101D4D00100244AC0080BB00090582094602010067
:081D5D00000725010100000050
:102B5A006173268243545553425F5461626C6530F7
:102B6A00312FC6F0826946690000000000000000AB
:102B7A00000000000000000000000000000000004B
:102B8A000000000000474F206C696E6B2032000085
:102B9A00000000000000000000000000000000002B
:102BAA0000000000006946692055534220417564BF
:102BBA00696F20534500000000000000000000007B
:102BCA000000000000474F206C696E6B2032000045
:102BDA0000000000000000000000000000000000EB
:102BEA000000000000474F206C696E6B2032000025
:102BFA0000000000000000000000000000000000CB
:102C0A000000000000474F206C696E6B2032000004
:102C1A0000000000000000000000000000000000AA
:102C2A0000000000006011474F206C696E6B203273
:102C3A002055414331000000000000000000000060
:102C4A0000000000000000474F206C696E6B2032C4
:102C5A002055414331000000000000000000000040
:102C6A0000000000000000474F206C696E6B2032A4
:102C7A002055414331000000000000000000000020
:102C8A0000000000000000474F206C696E6B203284
:102C9A002055414331000000000000000000000000
:102CAA0000000000000000474F206C696E6B203264
:102CBA0020554143310000000000000000000000E0
:072CCA000000000000000003
:05306000902801EFF0D3
:1030650064017BFF70067A1A793980047A1A794BE4
:10307500902808EBF0A3EAF0A3E9F01223F9FF90FA
:103085002804E4F0A3EFF0902868E0FFA3E090287F
:1030950006CFF0A3EFF0E4902802F0A3F090280407
:1030A500E0FEA3E0FF902802E0FCA3E0FDC39FEC57
:1030B5009E503B902868E0FEA3E07802C333CE33F0
:1030C500CED8F92DFFEC3EFE902808E0FBA3E0FAF0
:1030D500A3E0F98D828C83122412FD12607C902866
:1030E50003E004F070B7902802E004F080AF902868
:1030F50006E0FEA3E07802C333CE33CED8F9240828
:10310500FFE43EFE90268FA3E0FD12607C9028062A
:10311500E0FEA3E07802C333CE33CED8F92409FF0D
:10312500E43EFE90268FE0FD12607C902801E0646D
:1031350001703A902806E0FEA3E07802C333CE334F
:10314500CED8F9240AFFE43EFE902753A3E0FD12F2
:10315500607C902806E0FEA3E07802C333CE33CE30
:10316500D8F9240BFFE43EFE9027538038902806BB
:10317500E0FEA3E07802C333CE33CED8F9240AFFAC
:10318500E43EFE902691A3E0FD12607C902806E0C7
:10319500FEA3E07802C333CE33CED8F9240BFFE487
:1031A5003EFE902691E0FD12607C7D06E4FF1260F4
:1031B5006F902868A3E0FD7F1012606F902868E08B
:1031C500FD7F1112606F7B307D107F11125CC39003
:1031D5002805E02403FF902804E03400FEEF780280
:1031E500CEC313CE13D8F9FF902869E02FF09028AD
:0431F50068E03EF060
:0131F90022B3
:0716CA00902801EDF0AC07D0
:1016D100E0FE25E02418902804F0EEB40900400350
:1016E1000218059016EBF828287302170602172234
:1016F10002173202174F02176C0217890217A6024E
:1017010017CB0217E77BFF7A1A795D902805EBF07A
:10171100A3EAF0A3E9F01223F9FF902808E40218E4
:10172100019028057401F0A37426F0A374930217A5
:10173100C1EC64017B0170067A27795580047A2611
:1017410079B3902805EBF0A3EAF0A3E98072EC6489
:10175100017B0170067A27797580047A2679D39006
:101761002805EBF0A3EAF0A3E98055EC64017B01C5
:1017710070067A27799580047A2679F3902805EB0B
:10178100F0A3EAF0A3E98038EC64017B0170067AEA
:101791002779B580047A277913902805EBF0A3EA1D
:1017A100F0A3E9801BEC64017B0170067A2779D5EF
:1017B10080047A277933902805EBF0A3EAF0A3E9B6
:1017C100F0A3E4F0A37420F0803A90280574FFF0B0
:1017D100A3741AF0A3741DF07BFF7A1AF9125F86C5
:1017E100902808EE801A90280574FFF0A3741AF06F
:1017F100A3742BF07BFF7A1AF9125F86902808EE0A
:10180100F0A3EFF0902801E0FFD39400748094805E
:10181100500302196FD3EF9406748094805059E4F9
:10182100A3F0A3F0902802E0FEA3E0FFC39420EE12
:1018310064809480502D902805E0FBA3E0FAA3E09A
:10184100F9C3741F9FFFE49E8F82F58312241264F3
:10185100207010902803E004F070C9902802E00481
:10186100F080C1902802E0FEA3E0FFC3902809E0C8
:101871009FF0902808E09EF0902868E0FEA3E078B1
:1018810002C333CE33CED8F9FF902808A3E025E078
:101891002402FD12607C902868E0FEA3E07802C378
:1018A10033CE33CED8F92401FFE43EFE7D0312602E
:1018B1007CE4902802F0A3F0902808E0FEA3E0FF6A
:1018C100902802E0FCA3E0FDC39FEC9E40030219B7
:1018D10056902868E0FEA3E07802C333CE33CED819
:1018E100F92402FBE43EFAED25E0FFEC33FEEB2F99
:1018F100FFEA3EFE902805E0FBA3E0FAA3E0F990A1
:101901002802E0FCA3E0F5828C83122412FD126010
:101911007C902803E025E0FF902802E033FEEF24CD
:1019210001FDE43EFC902868E0FEA3E07802C333A9
:10193100CE33CED8F92402FFE43ECF2DCF3CFEE4D6
:10194100FD12607C902803E004F07006902802E00C
:1019510004F00218B9902809E025E0FF902808E07A
:1019610033FEEF2402FFE43EF0A3EFF08058E49051
:101971002802F0A3F0902808E0FEA3E0FF902802DF
:10198100E0FCA3E0FDC39FEC9E503B902868E0FE85
:10199100A3E07802C333CE33CED8F92DFFEC3EFE5F
:1019A100902805E0FBA3E0FAA3E0F98D828C831275
:1019B1002412FD12607C902803E004F070B7902897
:1019C10002E004F080AF7D06E4FF12606F9028040E
:1019D100E0FF902868A3E0FD12606F902804E00406
:1019E100FF902868E0FD12606F902804E004FF7BFF
:1019F100307D10125CC3902809E02403FF90280871
:101A0100E03400FEEF7802CEC313CE13D8F9FF9075
:0B1A11002869E02FF0902868E03EF00C
:011A1C0022A7
:102D17009028C7E090280630E016E4F0A374C4F0CA
:102D270090280174FFF0A3741AF0A37493F0801530
:102D37007401F0A37450F090280174FFF0A3741B82
:102D4700F0A37457F0902868E0FFA3E0902808CF1D
:102D5700F0A3EFF0E4FDFF12606FE4902804F0A306
:102D6700F0902806E0FEA3E0FF902804E0FCA3E033
:102D7700FDC39FEC9E503B902808E0FEA3E078023D
:102D8700C333CE33CED8F92DFFEC3EFE902801E0B9
:102D9700FBA3E0FAA3E0F98D828C83122412FD12C3
:102DA700607C902805E004F070B7902804E004F0F8
:102DB70080AF7D06E4FF12606F902808A3E0FD7FD7
:102DC7001212606F902808E0FD7F1312606F7B304E
:102DD7007D107F13125CC3902808A3E0FD7F1412B7
:102DE700606F902808E0FD7F1512606F7B307D10C3
:102DF7007F15125CC3902806E4F0A374BEF09028F8
:102E07000174FFF0A3741CF0A374A7F09028087452
:102E170007F0A374C0F0E4FDFF12606FE49028048C
:102E2700F0A3F0902806E0FEA3E0FF902804E0FC62
:102E3700A3E0FDC39FEC9E503B902808E0FEA3E073
:102E47007802C333CE33CED8F92DFFEC3EFE90285F
:102E570001E0FBA3E0FAA3E0F98D828C8312241230
:102E6700FD12607C902805E004F070B7902804E01C
:102E770004F080AF7D06E4FF12606F902808A3E09E
:102E8700FD7FA412606F902808E0FD7FA512606F98
:102E97007B307D107FA5125CC3902808A3E0FD7FDF
:102EA700A612606F902808E0FD7FA712606F7B3045
:072EB7007D107FA7025CC340
:1031FA007BFF7A1A7980902803EBF0A3EAF0A3E91F
:10320A00F01223F9FF902806E4F0A3EFF0E49028E7
:10321A0001F0A3F0902806E0FEA3E0FF902801E069
:10322A00FCA3E0FDC39FEC9E503B902868E0FEA300
:10323A00E07802C333CE33CED8F92DFFEC3EFE90B0
:10324A002803E0FBA3E0FAA3E0F98D828C83122421
:10325A0012FD12607C902802E004F070B7902801F9
:10326A00E004F080AF7D06E4FF12606F7D027F0606
:10327A0012606F902868A3E0FD7F0812606F9028A3
:10328A0068E0FD7F0912606F7B307D107F09125C58
:10329A00C3902807E02403FF902806E03400FEEFDD
:1032AA007802CEC313CE13D8F9FF902869E02FF025
:1032BA00902868E03EF0902806E4F0A3741FF0908E
:1032CA00280374FFF0A3741AF0A37461F0E4902841
:1032DA0001F0A3F0902806E0FEA3E0FF902801E0A9
:1032EA00FCA3E0FDC39FEC9E503B902868E0FEA340
:1032FA00E07802C333CE33CED8F92DFFEC3EFE90F0
:10330A002803E0FBA3E0FAA3E0F98D828C83122460
:10331A0012FD12607C902802E004F070B790280138
:10332A00E004F080AF902868A3E0FD7F0A12606F86
:10333A00902868E0FD7F0B12606F7B307D107F0B59
:10334A00125CC3902806A3E0FD7F0C12606F9028E0
:10335A0006E0FD7F0D12606F902807E02403FF90BE
:10336A002806E03400FEEF7802CEC313CE13D8F954
:0D337A00FF902869E02FF0902868E03EF0F9
:013387002223
:1044EA007BFF7A1A7989902803EBF0A3EAF0A3E913
:1044FA00F01223F9FF902806E4F0A3EFF0E49028E5
:10450A0001F0A3F0902806E0FEA3E0FF902801E066
:10451A00FCA3E0FDC39FEC9E503B902868E0FEA3FD
:10452A00E07802C333CE33CED8F92DFFEC3EFE90AD
:10453A002803E0FBA3E0FAA3E0F98D828C8312241E
:10454A0012FD12607C902802E004F070B7902801F6
:10455A00E004F080AF7D06E4FF12606F902868A344
:10456A00E0FD7FA212606F902868E0FD7FA31260D1
:10457A006F7B307D107FA3125CC3902807E0240371
:10458A00FF902806E03400FEEF7802CEC313CE1364
:0F459A00D8F9FF902869E02FF0902868E03EF0F4
:0145A90022EF
:102CD1004328EE0000004728E60000000000000045
:082CE1004128F1004128ED003B
:105CE6001252627DFF7FA7125EF07DFFE4FF125E17
:105CF600D57DFFE4FF125F0BE4FD7FA7125C9F02D8
:025D06005D0836
:105ED500904000E0FE7402F0EDF4FC90400AE05CB6
:0A5EE500FCEF5D4CF0904000EEF081
:015EEF002290
:105EF000904000E0FE7402F0EDF4FC904008E05C9D
:0A5F0000FCEF5D4CF0904000EEF065
:015F0A002274
:105C9F00904000E0FE7402F0904009E0FCEFF4FB4E
:105CAF00EC5BFCED6003EC4FFC904009ECF0904096
:035CBF0000EEF004
:015CC20022BF
:105F0B00904000E0FE7402F0EDF4FC90400FE05C7A
:0A5F1B00FCEF5D4CF0904000EEF04A
:015F25002259
:062CE90043290300000076
:105E9D00904000E09027FFF0E4FDFF12606F7F322D
:0B5EAD001260629027FFE0904000F0C0
:015EB80022C7
:105E8000904000E09027FDF07D02E4FF12606F7FFC
:0C5E9000131260629027FDE0904000F0CB
:015E9C0022E3
:105E4400904000E09027FDF0E4FDFF12606F7D02BA
:0D5E54007F4312606F9027FDE0904000F04A
:015E6100221E
:055BB800902809EFF048
:105BBD00904000E090280AF0E4FDFF12606F9028FD
:105BCD0009E0FD7B037F30125CC390280AE0904012
:025BDD0000F0D6
:015BDF0022A3
:105EB900904000E09027FFF0E4FDFF12606F7F3310
:0B5EC9001260629027FFE0904000F0A4
:015ED40022AB
:105D6B00904000E09027FFF0E4FDFF12606F7B0492
:0F5D7B007D047F30125CC39027FFE0904000F062
:015D8A0022F6
:105F5A00904000E09027FFF0E4FDFF12606F902769
:065F6A00FFE0904000F092
:015F7000220E
:104E7C00904000E09027FFF0E4FDFF12606F7DA4EE
:104E8C007F0112606F7D01E4FF12606F7B07E4FD10
:104E9C007F01125CC37D03E4FF12606F7BE07DE059
:104EAC007F02125CC37B087D087F1E125CC37D04ED
:104EBC00E4FF12606F7BE07DE07F02125CC37B0835
:104ECC007D087F1E125CC37D02E4FF12606F7B4085
:104EDC00E4FD7F18125CC37B807D807F18125CC35D
:084EEC009027FFE0904000F068
:014EF400229B
:1052C200904000E09027FFF07D01E4FF12606F7BC9
:1052D200077D027F01125CC37D03E4FF12606F7BD6
:1052E200E0E4FD7F02125CC37B08E4FD7F1E125CDA
:1052F200C37D04E4FF12606F7BE0E4FD7F02125C79
:10530200C37B08E4FD7F1E125CC3E4FDFF12606FE5
:0F5312007D207F0112606F9027FFE0904000F038
:015321002269
:10576E00C2AF124E7C904000E0FFE4800EEE54017A
:10577E006005ED64037013E4904000F0904033E058
:10578E00FE904032E0540FFD80E39040A8EDF0A370
:0C579E00EEF0904000EFF01252C2D2AFCB
:0157AA0022DC
:10566F009028C7E0C31330E0047F0380027F02124B
:10567F005BB8904000E0902808F07D01E4FF1260D5
:10568F006F7B077D027F01125CC3E4FDFF12606F29
:0F569F007D207F0112606F902808E0904000F09E
:0156AE0022D9
:1053E0009028C7E0C31330E0047F0180027F0012E1
:1053F0005BB8904000E0902808F07D01E4FF126067
:105400006F7B07E4FD7F01125CC3E4FDFF12606F58
:105410007DA47F0112606F7F321260967D02E4FFEF
:1054200012606F7B40E4FD7F18125CC37B807D803F
:0D5430007F18125CC3902808E0904000F047
:01543D00224C
:042CEF004129060071
:0400060000000022D4
:105B6600E4FF126062902802EFF07D0EE4FF1260FF
:105B76006F7D18E4FF125EF07D027F1112606F9058
:095B86002802E0FDE4FF02606F5B
:0760C4007DC07F1002606F38
:105F40007DA07F1012606FE4FFEFC39464748094AF
:095F50008050061200060F80F0DB
:015F59002225
:0760CB007D017F1402606FEC
:0760AD007F10126062EF1387
:0160B40022C9
:0D6039007F10126062EF54087002D322C382
:016046002237
:0F600C003003047D9080027D807F1012606F2230
:0760D2007D037F1402606FE3
:10594D00A202920312600C1260D2E4902850F0A3D0
:10595D00F01260AD401D902851E004F070069028C3
:10596D0050E004F0C3902851E094E8902850E09462
:08597D000340DE7F13026062AB
:03562E00A3E0FFF7
:05563100902850EFF08D
:105636001260CB902850E0FD7F1212606FE4902834
:1056460051F0A3F01260AD401D902852E004F070B6
:1056560006902851E004F0C3902852E094E8902880
:0956660051E0940340DE026039BA
:0B512D0090280EEEF0A3EFF0A3EDF0D1
:105138009028127405F0E4FF126062902811EFF0D5
:10514800D2007D0EE4FF12606F902812E0FF14F089
:10515800EF602F1260D9902906EFF01260C49028F2
:105168006AE0FF12563190280E12562E902810E051
:10517800FF12563100125F401260D9902906E0B53F
:0E51880007C7902811E0FDE4FF12606FA2003F
:0151960022F6
:084F6E0090280CEEF0A3EFF017
:104F76009028107405F0E4FF12606290280EEFF09E
:104F86007D0EE4FF12606F902810E0FF14F0EF60D2
:104F96003D1260D9902906EFF01260C490286AE0AD
:104FA600FF12563190280C12562E1260C490286AB1
:104FB600E04401FF125631D20212594D90280FEFEC
:104FC600F0125F401260D9902906E0B507B9902823
:0D4FD6000EE0FDE4FF12606F90280FE0FF79
:014FE30022AB
:0D5B8F0090280AEDF0A3EBF0902809EFF04C
:105B9C007E00124F6E90280BE0FDF45FFC902809FC
:0C5BAC00E0FF7E00A3E05D4CFD02512DE7
:0E434B00902808EFF0A3ECF0A3EDF0A3EBF048
:10435900E4FF126062902811EFF0D2007D0EE4FFB5
:1043690012606FE4902810F0902810E0C3940A744A
:10437900809480501A1260C4902808E0FF125631C8
:10438900400D7F01126096902810E004F080D990CA
:104399002810E0640A7004C200806BE4902810F0D1
:1043A900902810E0C3940A748094805025902809BD
:1043B900E0FF1256319200902809A3E0FF1256310E
:1043C900920020000D7F01126096902810E004F001
:1043D90080CE300031E490280FF090280BE0FF9058
:1043E900280FE0C39F501F90280CE0FBA3E475F051
:1043F900011224A9A9F0FA1223F9FF1256319028C3
:104409000FE004F080D4125F40902811E0FDE4FF32
:0544190012606FA2001B
:01441E00227B
:0E3AD200902846EFF0A3ECF0A3EDF0A3EBF08C
:103AE000D201E4FF12606290284FEFF07D0EE4FFF8
:103AF00012606FE490284EF090284EE0C3940A7450
:103B0000809480501A1260C4902846E0FF1256310B
:103B1000400D7F0112609690284EE004F080D9900D
:103B2000284EE0640A70028047902847E0FF125652
:103B300031902847A3E0FF125631E490284EF090D0
:103B4000284EE0C3940A74809480501C1260C49084
:103B50002846E04401FF125631400D7F0112609665
:103B600090284EE004F080D790284EE0640A70124E
:103B7000C201125F4090284FE0FDE4FF12606FA287
:103B80000122E490284DF0902849E0FF90284DE074
:103B9000FEC39F5033EF14B50604D2008002C2006A
:103BA000A200920212594D90284AE0FBA3E475F05E
:103BB000011224A9A9F0FAEF12243F7F01126096A6
:103BC00090284DE004F080BF125F4090284FE0FD48
:063BD000E4FF12606FD358
:013BD60022CC
:102CF3004128FA004128F7004228F400004128F94E
:062D0300004228F200006E
:105D0800E4FD7F80125C9F7F281260967D017F8072
:105D1800125C9F7F141260967D017F20125C9F02A7
:025D28004C4FDE
:0E601B009027FD7401F0125BE09028F7EFF083
:016029002254
:105F9B009028FAE0FDEF4E6004ED4401FD7F077E93
:045FAB000002512D72
:105DAA007F01EF600614600A14800D9028FA74C00F
:0E5DBA00F022E49028FAF0229028FA7418F0F3
:015DC80022B8
:1020360090286A7490F07D01E4FFFE12512D7F0610
:10204600126096E4FDFFFE12512D7F061260967D0A
:102056008C7F017E0012512D7D347F027E0012514D
:102066002D7D407F037E0012512D7D087F047E006A
:1020760012512D7D687F057E0012512D7D027F064F
:102086007E0012512DE4FD7F07FE12512D7DA97FA2
:10209600087E0012512D7D187F097E0012512D7D7C
:1020A600027F0A7E0012512D7D907F0B7E00125119
:1020B6002D7DAF7F0C7E0012512DE4FD7F0DFE12AB
:1020C600512D7D0A7F0E7E0012512D7DFF7F0F7EE2
:1020D6000012512D7DFF7F107E0012512D7DFF7F56
:1020E600117E0012512D7DFF7F127E0012512D7D33
:1020F600FF7F137E0012512D7D7F7F147E001251CB
:102106002D7D0D7F157E0012512DE4FD7F16FE12EA
:10211600512DE4FD7F17FE12512DE4FD7F18FE12AE
:10212600512DE4FD7F19FE12512D7D627F1A7E002E
:1021360012512D7DD47F1B7E0012512D7DF07F1C08
:102146007E0012512D7D047F1D7E0012512DE4FD6F
:102156007F1EFE12512DE4FD7F1FFE12512D7D1BA9
:102166007F207E0012512D7DFF7F217E0012512D92
:10217600E4FD7F22FE12512DE4FD7F23FE12512D38
:10218600E4FD7F24FE12512DE4FD7F25FE12512D24
:10219600E4FD7F26FE12512D7DCC7F277E00125155
:1021A6002DE4FD7F28FE12512DE4FD7F29FE1251FC
:1021B6002DE4FD7F2AFE12512DE4FD7F2BFE1251E8
:1021C6002DE4FD7F2CFE12512DE4FD7F2DFE1251D4
:1021D6002DE4FD7F2EFE12512DE4FD7F2FFE1251C0
:1021E6002D7D017F307E0012512D7D627F317E0074
:1021F60012512D7DC07F327E0012512D7D0D7F3311
:102206007E0012512D7D627F347E0012512DE4FD39
:102216007F35FE12512DE4FD7F36FE12512DE4FD71
:102226007F37FE12512DE4FD7F38FE12512DE4FD5D
:102236007F92FE12512D7D017F937E0012512D7DDE
:10224600807F957E0012512D125DAA9028FAE0FD3E
:102256007F077E0012512D7D117F887E0012512D41
:102266007DFF7F897E0012512D7D547F8A7E00126C
:10227600512D7DFF7F8B7E0012512D7D547F8C7EEC
:102286000012512D7D507F8D7E0012512D7D1C7FB9
:102296008E7E0012512D7DB97F8F7E0012512D7DCD
:1022A600517F907E0012512D7D0F7F917E0012513D
:1022B6002D7DD17F167E0012512DE4FD7F17FE1273
:1022C600512D7D907F187E0012512DE4FD7F19FE61
:1022D60012512DE4FD7F80FE12512D7D5F7F827E9F
:1022E6000012512DE4FD7F83FE12512D7D5F7F8408
:0D22F6007E0012512DE4FD7F85FE02512D6A
:0F602A00125DAA9028FAE0FD7F077E0002512D3B
:0E6047007D017F20125C9FE4FD7F80025C9F44
:105E6200125B667D017F80125C9F7D017F20125C48
:0E5E72009F7FC81260961220367F64026096F1
:105DC9007FC812609612601B9028F7E060051220C8
:0F5DD900368007E4FD7F80125C9F7F6402609636
:104EF5009028F7E0607290286A7490F0EF60227D48
:104F0500017F20125C9F7B017D017F07125B8F7DF6
:104F1500FF7F0F7E0012512D7DFF7F107E00025115
:104F25002D902901E060417F641260967B01E4FDCC
:104F35007F07125B8F9028FFE0FFA3E0FD125D2A3B
:104F4500E4FD7F20125C9F9028C2E06401701490FC
:104F550040007403F07F18126062EF5408FF60038D
:084F65001258617F641260968E
:014F6D002221
:105055009028F7E0606690286A7490F0EF24F85085
:1050650007602614602380457D027F0A7E00125169
:105075002D7D6B7F0C7E0012512D7D407F037E00C0
:1050850012512D7B08E4FD801F7D027F0A7E0012F0
:10509500512D7DBB7F0C7E0012512D7D417F037EFE
:1050A5000012512D7B087D087F07125B8F7D807F65
:0D50B500927E0012512D9028F87401F02217
:10551C009028F7E0603E90286A7490F0EF24FC50DD
:10552C000280247D027F0A7E0012512D7D6B7F0C40
:10553C007E0012512D7D407F037E0012512D7B0881
:10554C00E4FD7F07125B8FE4FD7F92FE12512DE488
:05555C009028F8F02288
:105561009028F7E0603E90286A7490F0EF24FC5098
:105571000280247D027F0A7E0012512D7D6B7F0CFB
:105581007E0012512D7D407F037E0012512D7B083C
:10559100E4FD7F07125B8FE4FD7F92FE12512DE443
:0555A1009028F8F02243
:105D2A0090280DEDF09028F7E06015AD077F0F7E03
:105D3A000012512D90280DE0FD7F107E0012512D8A
:015D4A002236
:0160F7002286
:0160F8002285
:10000E007D017F01125C9FE4FD7F02125C9F7D01EA
:05001E007F04025C9F5D
:104C4F009028F6E07003024CE3E4F0902901E012A3
:104C5F0025334C9E004C9E104C9E114C9E124C9E28
:104C6F00134CA2144CA2154CA2164CA2174CA2180E
:104C7F004CA2194CB4204CB4214CC6224CC6234C28
:104C8F00B4404CB4414CC6424CC64300004CDB7D93
:104C9F00018002E4FD7F01125C9FE4FD7F02125C44
:104CAF009F7D0180227D017F01125C9FE4FD7F02C9
:104CBF00125C9FE4FD80107D017F01125C9F7D01DE
:104CCF007F02125C9FE4FD7F04125C9F902901E03C
:054CDF00FF1259F22252
:104BB8009028F7E07003024C4E90286A7490F07FBA
:104BC800487E00124F6E9027FDEFF07F417E001265
:104BD8004F6EEF54F0FF9027FDE054C0F07003EFE4
:104BE8006007E49028F2F0A3F09028F2E0FEA3E03A
:104BF800FFC39432EE64809480504BEF4E7017FDE3
:104C08007F0BFE12512D7D907F0B7E0012512D7F60
:104C1800017E00125F9B9028F3E004F07006902854
:104C2800F2E004F09028F2E07004A3E06432701619
:104C3800FD7F0BFE12512D7D907F0B7E0012512DB2
:064C4800E4FFFE125F9B79
:014C4E002243
:0D2D09004228FF000041290100412902007D
:0360E500025DC990
:105FD600AE07EF4410902901F09028F67401F00204
:025FE600505514
:105FE800AE07EF4420902901F09028F67401F002E2
:025FF800551C36
:105FFA00AE07EF4440902901F09028F67401F002B0
:02600A005561DE
:0360E800025D2A2C
:0860B500902902EFF0024EF504
:0360EB000260E56B
:0360EE000260F756
:0360F1000260F852
:10338800636D643A7374726D2C76616C3A257800BB
:10339800636D643A6765745F616C6C2C6D5F7479FA
:1033A80070653A676F6C6B322C7665723A25642EBD
:1033B80025642C766F6C3A25642C666C743A256407
:1033C8002C7374726D3A257800636D643A666C7478
:1033D8002C76616C3A256400636D643A766F6C2CC8
:1033E80076616C3A256400007D007C007B007900E2
:1033F80078007700760074007300720070006F0028
:103408006E006D006B006A00690067006600650069
:1034180064006200610060005F005D005C005B00AA
:1034280059005800570056005400530052005100EC
:103438004F004E004D004B004A004900480046002E
:10344800450044004300410040003F003D003C006F
:103458003B003A00380037003600350033003200B0
:10346800310030002E002D002C002A0029002800F1
:103478002700250024002300220020001F001E0032
:103488001D001B001A001900170016001500140073
:103498001200110010000F000D000C000B000A00B4
:1034A80008000700060005000300020001000000F4
:1034B8000000000000000000000000000000000004
:1034C80000000000000000000000000000000000F4
:1034D80000000000000000000000000000000000E4
:0F34E800000000000000000000000000000000D5
:10589D00902801EEF0A3EFF0A3EBF0A3EAF0A3E95B
:0358AD00F0AF0554
:1058B000902801E0FCA3E0FDAB07A3E0F9A3E0FA28
:1058C000A3E090280CC9F0A3EAF0A3E9F07FA012AE
:0858D000434BE433902806F07D
:0158D80022AD
:06572F007B017D017E00FC
:10573500902841EEF0A3EFF0A3EBF0A3EAF0A3E984
:03574500F0AF05BD
:10574800902841E0FCA3E0FDAB07A3E0F9A3E0FA51
:10575800A3E090284AC9F0A3EAF0A3E9F07FA012D9
:055768003AD2E433FF1A
:01576D002219
:105F71009027FF74F1F07B017A2779FF7D017F2063
:055F81007E0002589DA6
:105BE0007A2779FE7F2012572FEF7002FF2290272D
:105BF000FEE0F47005125F71800B9027FEE064F107
:075C000060037F00227F0119
:015C0700227A
:105FAF00902800EFF07B017A2879007D017F017E38
:045FBF000002589DE7
:105DE8007A2879407F0112572F902840E0D39402F7
:0E5DF8007480948040037401F0902840E0FF16
:015E06002279
:1056AF009040007406F07D0B7FE512606F7DB07F38
:1056BF00E412606F7D3B7F0F12606F7D407FE012C1
:1056CF00606F7DC07FE112606F7DA07FE212606F1F
:1056DF007D037FE312606F7B037D037FE6025CC374
:105AE400E4FFEFC3946474809480501F9028FFE017
:105AF400FDEF25E024EFF582E43433F583D374011C
:0B5B0400939DE493940040030F80D7B2
:015B0F002273
:0654D6007B01AD07AC06EE
:1054DC00ED540FFFC374109F902841F0E4902840C6
:1054EC00F0902841E0FF902840E0FEC39F5017EE5B
:1054FC007E002DF582EE3CF58374FF12245190282A
:0F550C0040E004F080DB902841E02DFFE43CFEFE
:01551B00226D
:1059F20090284374FFF0A37433F0A37488F0A3E4F7
:105A0200F0A3EFF07B017A2779FF1213CAD3EF9448
:105A120000EE64809480400C7A2779FF1254D6AD50
:045A2200071255A66C
:015A2600225D
:104DFD0078FF7C277D017BFF7A3479B77E007F4079
:104E0D001223D3125AE490283FEFF0125DE8902858
:104E1D004374FFF0A37433F0A37498F0A3E4F0A3EC
:104E2D0004F0A3E4F0A37417F090283FE0FC339551
:104E3D00E090284AF0A3CCF0EF3395E0A3F0A3EF78
:104E4D00F0902901E0FF90284EE4F0A3EFF07B01F4
:104E5D007A2779FF1213CAD3EF9400EE6480948001
:0E4E6D00400C7A2779FF1254D6AD071255A6D5
:014E7B002214
:1057AB00125DE890284374FFF0A37433F0A374D117
:1057BB00F0EF3395E0A3F0A3EFF07B017A2779FFAD
:1057CB001213CAD3EF9400EE64809480400E7B01D9
:0C57DB007A2779FF1254D8AD071255A6AA
:0157E700229F
:1057E800125AE490284374FFF0A37433F0A374E0D2
:1057F800F0EF3395E0A3F0A3EFF07B017A2779FF70
:105808001213CAD3EF9400EE64809480400E7B019B
:0C5818007A2779FF1254D8AD071255A66C
:015824002261
:105E0700EF25E024EFF582E43433F583740193FE44
:0F5E17009028FFF0A3F0FD9028FFE0FF025D2A26
:1056EF009027FFEDF0EFC39406748094805030EF55
:1056FF0024FD6023240270279028F9E0600E125ECB
:10570F0062E49028F9F09028F4F0A3F09027FFE0DE
:10571F00FF125FAF02602A9027FFE0FF125E0722A1
:105B1000EFC39406748094805021EF24FE600E241D
:105B2000FE600D14600D24057011024DFD0257AB8F
:0C5B30000257E8902901E0FF1259F22210
:03000000024D713D
:0C4D7100787FE4F6D8FD758121024DB872
:10230300E709F608DFFA8046E709F208DFFA803EBC
:1023130088828C83E709F0A3DFFA8032E309F608A9
:10232300DFFA8078E309F208DFFA807088828C8311
:10233300E309F0A3DFFA806489828A83E0A3F608C5
:10234300DFFA805889828A83E0A3F208DFFA804C9F
:1023530080D280FA80C680D4806980F28033801076
:1023630080A680EA809A80A880DA80E280CA8033DF
:1023730089828A83ECFAE493A3C8C582C8CCC58357
:10238300CCF0A3C8C582C8CCC583CCDFE9DEE78027
:102393000D89828A83E493A3F608DFF9ECFAA9F0A6
:1023A300EDFB2289828A83ECFAE0A3C8C582C8CCFC
:1023B300C583CCF0A3C8C582C8CCC583CCDFEADE15
:1023C300E880DB89828A83E493A3F208DFF980CC77
:1023D30088F0EF60010E4E60C388F0ED2402B40470
:1023E3000050B9F582EB2402B4040050AF23234517
:0623F300822390235373C6
:1023F900BB010689828A83E0225002E722BBFE02E2
:09240900E32289828A83E4932214
:10241200BB010CE58229F582E5833AF583E022507F
:1024220006E92582F8E622BBFE06E92582F8E222C9
:0D243200E58229F582E5833AF583E49322E3
:10243F00BB010689828A83F0225002F722BBFE017C
:02244F00F32276
:10245100F8BB010DE58229F582E5833AF583E8F0C1
:10246100225006E92582C8F622BBFE05E92582C86D
:02247100F22255
:10247300C2D5EC30E709B2D5E4C39DFDE49CFCEE84
:1024830030E715B2D5E4C39FFFE49EFE122559C37E
:10249300E49DFDE49CFC800312255930D507C3E479
:0624A3009FFFE49EFE22F3
:1024A900A3F8E0C5F025F0F0E582158270021583E6
:0624B900E0C838F0E82243
:1024BF00EB9FF5F0EA9E42F0E99D42F0E89C45F073
:0124CF0022EA
:1024D000E8600FECC313FCED13FDEE13FEEF13FFEA
:0324E000D8F1220E
:1024E300E8600FEFC333FFEE33FEED33FDEC33FC57
:0324F300D8F122FB
:0C24F600ECF0A3EDF0A3EEF0A3EFF02259
:10250200A8828583F0D083D0821225191225191250
:102512002519122519E473E493A3C583C5F0C58375
:10252200C8C582C8F0A3C583C5F0C583C8C582C823
:012532002286
:10253300D083D082F8E4937012740193700DA3A337
:1025430093F8740193F5828883E47374029368604B
:06255300EFA3A3A380DF4B
:10136500E5082443F582E43428F583E00508229056
:101375002840300703902843E475F0011225AE029A
:1013850023F92000E97F2ED2008018EF540F249016
:10139500D43440D4FF30040BEF24BFB41A005003FB
:1013A5002461FFE50960021509050CE50C700205CD
:1013B5000B30070E902840E475F0011225AEEF02C0
:1013C500243F025C2F7403D2078003E4C207F508AB
:1013D5009028401225C5E4F509F50BF50CE50960E3
:1013E500077F201213A880F5750AFFC201C200C24B
:1013F50002C203C205C206C208121374FF700D3083
:1014050007057F001213B9AF0CAE0B22B4255FC2DE
:10141500D5C204121374FF24D0B40A00501A75F013
:101425000A780930D50508B6FF0106C6A426F620B8
:10143500D5047002D20380D924CFB41A00EF50042A
:10144500C2E5D2040215BAD20180C6D20080C0D24C
:101455000280BCD2D580BAD20580B47F201213A8F1
:101465002002077401B5090040F1121365FF12133C
:10147500A80213E2D208D2068095121365FB121357
:1014850065FA121365F94A4B7006798B7A167BFF5C
:1014950020022EE509602A7E008E827583001224C3
:1014A5001260060EEE650A70F0C2D5EBC0E0EAC028
:1014B500E0E9C0E0EE121601D0E0F9D0E0FAD0E0A4
:1014C500FB1223F9FF60AAEBC0E0EAC0E0E9C0E047
:1014D5001213A8D0E02401F9D0E03400FAD0E0FBE3
:1014E500E50A0460DCD50AD980877BFF7A1579FD8A
:1014F500D202809C791080027908C206C208800851
:10150500D2D5790A8004790AC2D5E50A047002F5B4
:101515000AE4FAFDFEFF121365FC7B082001131295
:101525001365FD7B1030000A121365FE121365FF6B
:101535007B20EC3382D592D55013C3E43000069F4F
:10154500FFE49EFEE42001039DFDE49CFCE4CBF852
:10155500C201EC700CCFCECDCCE824F8F870F38046
:1015650017C3EF33FFEE33FEED33FDEC33FCEB3306
:10157500FB994002FB0FD8E9EB300105F8D0E0C438
:1015850048B201C0E00AEC4D4E4F78207B0070C296
:10159500EAB50A0040BCC0E0121603D0F0D0E02046
:1015A5000104C4C0E0C4B201C0F0121391D0F0D55B
:1015B500F0EB0213E2122533147F5314F95814503B
:1015C5004C144C4214FD4F1505441505491465434B
:0815D500150B5514EF4614EF4D
:1015DD004514EF4716AB5014542D14582E147B2B75
:1015ED00145C2314792016942A14144800001473E3
:1015FD003F3F3F00790AA2D5200314300509B910E9
:10160D00020404B9080104A2D520060250010420E9
:10161D0002689202B509005034C0E07F20300319F2
:10162D007F30A20272067205500F12165AC202C204
:10163D0006C205C2087F30800F300503E9C0E012F5
:10164D0013A8300503D0E0F9D0E0B509CC3005176B
:10165D007F30B9100C1213A87F583004077F7880A3
:10166D0003B908031213A83002057F2D0213A87FBA
:10167D00202008F87F2B2006F322920280CF286EBF
:10168D00756C6C2900D2011213653001F8C2017816
:10169D000930D50108F60214142D50434958121380
:1016AD00652403B405004001E49016A69312139926
:0D16BD00743A121399D2037509040214F94E
:105F8600E4FFFE1223F9600C0FEF70010E09E970B1
:055F9600F20A80EF2279
:104D7D00025381E493A3F8E493A34003F68001F278
:104D8D0008DFF48029E493A3F85407240CC8C33337
:104D9D00C4540F4420C8834004F456800146F6DF06
:104DAD00E4800B0102040810204080902AC9E47EA3
:104DBD00019360BCA3FF543F30E509541FFEE493FB
:104DCD00A360010ECF54C025E060A840B8E493A3C2
:104DDD00FAE493A3F8E493A3C8C582C8CAC583CAED
:104DED00F0A3C8C582C8CAC583CADFE9DEE780BEA5
:012D160000BC
:10255900BC000BBE0029EF8DF084FFADF022E4CC66
:10256900F875F008EF2FFFEE33FEEC33FCEE9DEC2F
:10257900984005FCEE9DFE0FD5F0E9E4CEFD22ED75
:10258900F8F5F0EE8420D21CFEADF075F008EF2FBF
:10259900FFED33FD4007985006D5F0F222C398FDB0
:0525A9000FD5F0EA224D
:1025AE00F8E0FBA3A3E0F925F0F0E58215827002B6
:0725BE001583E0FA38F0225A
:0925C500EBF0A3EAF0A3E9F02217
:105C2F00EFB40A07740D125C3A740A309811A899F0
:105C3F00B8130CC2983098FDA899C298B811F630D5
:075C4F0099FDC299F59922AD
:00000001FF
